Archive member included to satisfy reference by file (symbol)

d:/stm32cubeide_1.5.0/stm32cubeide/plugins/com.st.stm32cube.ide.mcu.externaltools.gnu-tools-for-stm32.7-2018-q2-update.win32_1.5.0.202011040924/tools/bin/../lib/gcc/arm-none-eabi/7.3.1/../../../../arm-none-eabi/lib/thumb/v7e-m/fpv4-sp/hard\libc_nano.a(lib_a-errno.o)
                              Core/Src/syscalls.o (__errno)
d:/stm32cubeide_1.5.0/stm32cubeide/plugins/com.st.stm32cube.ide.mcu.externaltools.gnu-tools-for-stm32.7-2018-q2-update.win32_1.5.0.202011040924/tools/bin/../lib/gcc/arm-none-eabi/7.3.1/../../../../arm-none-eabi/lib/thumb/v7e-m/fpv4-sp/hard\libc_nano.a(lib_a-exit.o)
                              d:/stm32cubeide_1.5.0/stm32cubeide/plugins/com.st.stm32cube.ide.mcu.externaltools.gnu-tools-for-stm32.7-2018-q2-update.win32_1.5.0.202011040924/tools/bin/../lib/gcc/arm-none-eabi/7.3.1/../../../../arm-none-eabi/lib/thumb/v7e-m/fpv4-sp/hard/crt0.o (exit)
d:/stm32cubeide_1.5.0/stm32cubeide/plugins/com.st.stm32cube.ide.mcu.externaltools.gnu-tools-for-stm32.7-2018-q2-update.win32_1.5.0.202011040924/tools/bin/../lib/gcc/arm-none-eabi/7.3.1/../../../../arm-none-eabi/lib/thumb/v7e-m/fpv4-sp/hard\libc_nano.a(lib_a-impure.o)
                              d:/stm32cubeide_1.5.0/stm32cubeide/plugins/com.st.stm32cube.ide.mcu.externaltools.gnu-tools-for-stm32.7-2018-q2-update.win32_1.5.0.202011040924/tools/bin/../lib/gcc/arm-none-eabi/7.3.1/../../../../arm-none-eabi/lib/thumb/v7e-m/fpv4-sp/hard\libc_nano.a(lib_a-exit.o) (_global_impure_ptr)
d:/stm32cubeide_1.5.0/stm32cubeide/plugins/com.st.stm32cube.ide.mcu.externaltools.gnu-tools-for-stm32.7-2018-q2-update.win32_1.5.0.202011040924/tools/bin/../lib/gcc/arm-none-eabi/7.3.1/../../../../arm-none-eabi/lib/thumb/v7e-m/fpv4-sp/hard\libc_nano.a(lib_a-init.o)
                              d:/stm32cubeide_1.5.0/stm32cubeide/plugins/com.st.stm32cube.ide.mcu.externaltools.gnu-tools-for-stm32.7-2018-q2-update.win32_1.5.0.202011040924/tools/bin/../lib/gcc/arm-none-eabi/7.3.1/../../../../arm-none-eabi/lib/thumb/v7e-m/fpv4-sp/hard/crt0.o (__libc_init_array)
d:/stm32cubeide_1.5.0/stm32cubeide/plugins/com.st.stm32cube.ide.mcu.externaltools.gnu-tools-for-stm32.7-2018-q2-update.win32_1.5.0.202011040924/tools/bin/../lib/gcc/arm-none-eabi/7.3.1/../../../../arm-none-eabi/lib/thumb/v7e-m/fpv4-sp/hard\libc_nano.a(lib_a-memcpy-stub.o)
                              Middlewares/Third_Party/FreeRTOS/Source/CMSIS_RTOS_V2/cmsis_os2.o (memcpy)
d:/stm32cubeide_1.5.0/stm32cubeide/plugins/com.st.stm32cube.ide.mcu.externaltools.gnu-tools-for-stm32.7-2018-q2-update.win32_1.5.0.202011040924/tools/bin/../lib/gcc/arm-none-eabi/7.3.1/../../../../arm-none-eabi/lib/thumb/v7e-m/fpv4-sp/hard\libc_nano.a(lib_a-memset.o)
                              d:/stm32cubeide_1.5.0/stm32cubeide/plugins/com.st.stm32cube.ide.mcu.externaltools.gnu-tools-for-stm32.7-2018-q2-update.win32_1.5.0.202011040924/tools/bin/../lib/gcc/arm-none-eabi/7.3.1/../../../../arm-none-eabi/lib/thumb/v7e-m/fpv4-sp/hard/crt0.o (memset)
d:/stm32cubeide_1.5.0/stm32cubeide/plugins/com.st.stm32cube.ide.mcu.externaltools.gnu-tools-for-stm32.7-2018-q2-update.win32_1.5.0.202011040924/tools/bin/../lib/gcc/arm-none-eabi/7.3.1/thumb/v7e-m/fpv4-sp/hard\libgcc.a(_arm_addsubdf3.o)
                              Core/Src/printf.o (__aeabi_dsub)
d:/stm32cubeide_1.5.0/stm32cubeide/plugins/com.st.stm32cube.ide.mcu.externaltools.gnu-tools-for-stm32.7-2018-q2-update.win32_1.5.0.202011040924/tools/bin/../lib/gcc/arm-none-eabi/7.3.1/thumb/v7e-m/fpv4-sp/hard\libgcc.a(_arm_muldivdf3.o)
                              Core/Src/printf.o (__aeabi_dmul)
d:/stm32cubeide_1.5.0/stm32cubeide/plugins/com.st.stm32cube.ide.mcu.externaltools.gnu-tools-for-stm32.7-2018-q2-update.win32_1.5.0.202011040924/tools/bin/../lib/gcc/arm-none-eabi/7.3.1/thumb/v7e-m/fpv4-sp/hard\libgcc.a(_arm_cmpdf2.o)
                              Core/Src/printf.o (__aeabi_dcmpeq)
d:/stm32cubeide_1.5.0/stm32cubeide/plugins/com.st.stm32cube.ide.mcu.externaltools.gnu-tools-for-stm32.7-2018-q2-update.win32_1.5.0.202011040924/tools/bin/../lib/gcc/arm-none-eabi/7.3.1/thumb/v7e-m/fpv4-sp/hard\libgcc.a(_arm_fixdfsi.o)
                              Core/Src/printf.o (__aeabi_d2iz)
d:/stm32cubeide_1.5.0/stm32cubeide/plugins/com.st.stm32cube.ide.mcu.externaltools.gnu-tools-for-stm32.7-2018-q2-update.win32_1.5.0.202011040924/tools/bin/../lib/gcc/arm-none-eabi/7.3.1/thumb/v7e-m/fpv4-sp/hard\libgcc.a(_arm_fixunsdfsi.o)
                              Core/Src/printf.o (__aeabi_d2uiz)
d:/stm32cubeide_1.5.0/stm32cubeide/plugins/com.st.stm32cube.ide.mcu.externaltools.gnu-tools-for-stm32.7-2018-q2-update.win32_1.5.0.202011040924/tools/bin/../lib/gcc/arm-none-eabi/7.3.1/thumb/v7e-m/fpv4-sp/hard\libgcc.a(_arm_truncdfsf2.o)
                              Core/Src/bmp280.o (__aeabi_d2f)
d:/stm32cubeide_1.5.0/stm32cubeide/plugins/com.st.stm32cube.ide.mcu.externaltools.gnu-tools-for-stm32.7-2018-q2-update.win32_1.5.0.202011040924/tools/bin/../lib/gcc/arm-none-eabi/7.3.1/thumb/v7e-m/fpv4-sp/hard\libgcc.a(_aeabi_uldivmod.o)
                              Core/Src/printf.o (__aeabi_uldivmod)
d:/stm32cubeide_1.5.0/stm32cubeide/plugins/com.st.stm32cube.ide.mcu.externaltools.gnu-tools-for-stm32.7-2018-q2-update.win32_1.5.0.202011040924/tools/bin/../lib/gcc/arm-none-eabi/7.3.1/thumb/v7e-m/fpv4-sp/hard\libgcc.a(_udivmoddi4.o)
                              d:/stm32cubeide_1.5.0/stm32cubeide/plugins/com.st.stm32cube.ide.mcu.externaltools.gnu-tools-for-stm32.7-2018-q2-update.win32_1.5.0.202011040924/tools/bin/../lib/gcc/arm-none-eabi/7.3.1/thumb/v7e-m/fpv4-sp/hard\libgcc.a(_aeabi_uldivmod.o) (__udivmoddi4)
d:/stm32cubeide_1.5.0/stm32cubeide/plugins/com.st.stm32cube.ide.mcu.externaltools.gnu-tools-for-stm32.7-2018-q2-update.win32_1.5.0.202011040924/tools/bin/../lib/gcc/arm-none-eabi/7.3.1/thumb/v7e-m/fpv4-sp/hard\libgcc.a(_dvmd_tls.o)
                              d:/stm32cubeide_1.5.0/stm32cubeide/plugins/com.st.stm32cube.ide.mcu.externaltools.gnu-tools-for-stm32.7-2018-q2-update.win32_1.5.0.202011040924/tools/bin/../lib/gcc/arm-none-eabi/7.3.1/thumb/v7e-m/fpv4-sp/hard\libgcc.a(_aeabi_uldivmod.o) (__aeabi_ldiv0)

Allocating common symbols
Common symbol       size              file

TimerBmpDataHandle  0x4               Core/Src/freertos.o
SemaphoreBmpQueueHandle
                    0x4               Core/Src/freertos.o
hi2c1               0x54              Core/Src/i2c.o
htim10              0x40              Core/Src/stm32f4xx_hal_timebase_tim.o
font                0x4               Core/Src/GFX_BW.o
OledTaskHandle      0x4               Core/Src/freertos.o
uwTick              0x4               Drivers/STM32F4xx_HAL_Driver/Src/stm32f4xx_hal.o
xQueueRegistry      0x40              Middlewares/Third_Party/FreeRTOS/Source/queue.o
pFlash              0x20              Drivers/STM32F4xx_HAL_Driver/Src/stm32f4xx_hal_flash.o
QueueBmpDataHandle  0x4               Core/Src/freertos.o
MutexPrintfHandle   0x4               Core/Src/freertos.o
oled_i2c            0x4               Core/Src/SSD1306_OLED.o
MutexI2C1Handle     0x4               Core/Src/freertos.o
Bmp280TaskHandle    0x4               Core/Src/freertos.o
MutexBmpDataHandle  0x4               Core/Src/freertos.o
huart2              0x40              Core/Src/usart.o
HeartbeatTaskHandle
                    0x4               Core/Src/freertos.o

Discarded input sections

 .text          0x0000000000000000        0x0 d:/stm32cubeide_1.5.0/stm32cubeide/plugins/com.st.stm32cube.ide.mcu.externaltools.gnu-tools-for-stm32.7-2018-q2-update.win32_1.5.0.202011040924/tools/bin/../lib/gcc/arm-none-eabi/7.3.1/thumb/v7e-m/fpv4-sp/hard/crti.o
 .data          0x0000000000000000        0x0 d:/stm32cubeide_1.5.0/stm32cubeide/plugins/com.st.stm32cube.ide.mcu.externaltools.gnu-tools-for-stm32.7-2018-q2-update.win32_1.5.0.202011040924/tools/bin/../lib/gcc/arm-none-eabi/7.3.1/thumb/v7e-m/fpv4-sp/hard/crti.o
 .bss           0x0000000000000000        0x0 d:/stm32cubeide_1.5.0/stm32cubeide/plugins/com.st.stm32cube.ide.mcu.externaltools.gnu-tools-for-stm32.7-2018-q2-update.win32_1.5.0.202011040924/tools/bin/../lib/gcc/arm-none-eabi/7.3.1/thumb/v7e-m/fpv4-sp/hard/crti.o
 .data          0x0000000000000000        0x4 d:/stm32cubeide_1.5.0/stm32cubeide/plugins/com.st.stm32cube.ide.mcu.externaltools.gnu-tools-for-stm32.7-2018-q2-update.win32_1.5.0.202011040924/tools/bin/../lib/gcc/arm-none-eabi/7.3.1/thumb/v7e-m/fpv4-sp/hard/crtbegin.o
 .text          0x0000000000000000       0x74 d:/stm32cubeide_1.5.0/stm32cubeide/plugins/com.st.stm32cube.ide.mcu.externaltools.gnu-tools-for-stm32.7-2018-q2-update.win32_1.5.0.202011040924/tools/bin/../lib/gcc/arm-none-eabi/7.3.1/../../../../arm-none-eabi/lib/thumb/v7e-m/fpv4-sp/hard/crt0.o
 .data          0x0000000000000000        0x0 d:/stm32cubeide_1.5.0/stm32cubeide/plugins/com.st.stm32cube.ide.mcu.externaltools.gnu-tools-for-stm32.7-2018-q2-update.win32_1.5.0.202011040924/tools/bin/../lib/gcc/arm-none-eabi/7.3.1/../../../../arm-none-eabi/lib/thumb/v7e-m/fpv4-sp/hard/crt0.o
 .bss           0x0000000000000000        0x0 d:/stm32cubeide_1.5.0/stm32cubeide/plugins/com.st.stm32cube.ide.mcu.externaltools.gnu-tools-for-stm32.7-2018-q2-update.win32_1.5.0.202011040924/tools/bin/../lib/gcc/arm-none-eabi/7.3.1/../../../../arm-none-eabi/lib/thumb/v7e-m/fpv4-sp/hard/crt0.o
 .ARM.extab     0x0000000000000000        0x0 d:/stm32cubeide_1.5.0/stm32cubeide/plugins/com.st.stm32cube.ide.mcu.externaltools.gnu-tools-for-stm32.7-2018-q2-update.win32_1.5.0.202011040924/tools/bin/../lib/gcc/arm-none-eabi/7.3.1/../../../../arm-none-eabi/lib/thumb/v7e-m/fpv4-sp/hard/crt0.o
 .ARM.exidx     0x0000000000000000        0x8 d:/stm32cubeide_1.5.0/stm32cubeide/plugins/com.st.stm32cube.ide.mcu.externaltools.gnu-tools-for-stm32.7-2018-q2-update.win32_1.5.0.202011040924/tools/bin/../lib/gcc/arm-none-eabi/7.3.1/../../../../arm-none-eabi/lib/thumb/v7e-m/fpv4-sp/hard/crt0.o
 .ARM.attributes
                0x0000000000000000       0x20 d:/stm32cubeide_1.5.0/stm32cubeide/plugins/com.st.stm32cube.ide.mcu.externaltools.gnu-tools-for-stm32.7-2018-q2-update.win32_1.5.0.202011040924/tools/bin/../lib/gcc/arm-none-eabi/7.3.1/../../../../arm-none-eabi/lib/thumb/v7e-m/fpv4-sp/hard/crt0.o
 .group         0x0000000000000000        0xc Core/Src/GFX_BW.o
 .group         0x0000000000000000        0xc Core/Src/GFX_BW.o
 .group         0x0000000000000000        0xc Core/Src/GFX_BW.o
 .group         0x0000000000000000        0xc Core/Src/GFX_BW.o
 .group         0x0000000000000000        0xc Core/Src/GFX_BW.o
 .group         0x0000000000000000        0xc Core/Src/GFX_BW.o
 .group         0x0000000000000000        0xc Core/Src/GFX_BW.o
Memory Configuration

Name             Origin             Length             Attributes
RAM              0x0000000020000000 0x0000000000020000 xrw
FLASH            0x0000000008000000 0x0000000000080000 xr
*default*        0x0000000000000000 0xffffffffffffffff

Linker script and memory map

LOAD d:/stm32cubeide_1.5.0/stm32cubeide/plugins/com.st.stm32cube.ide.mcu.externaltools.gnu-tools-for-stm32.7-2018-q2-update.win32_1.5.0.202011040924/tools/bin/../lib/gcc/arm-none-eabi/7.3.1/thumb/v7e-m/fpv4-sp/hard/crti.o
LOAD d:/stm32cubeide_1.5.0/stm32cubeide/plugins/com.st.stm32cube.ide.mcu.externaltools.gnu-tools-for-stm32.7-2018-q2-update.win32_1.5.0.202011040924/tools/bin/../lib/gcc/arm-none-eabi/7.3.1/thumb/v7e-m/fpv4-sp/hard/crtbegin.o
LOAD d:/stm32cubeide_1.5.0/stm32cubeide/plugins/com.st.stm32cube.ide.mcu.externaltools.gnu-tools-for-stm32.7-2018-q2-update.win32_1.5.0.202011040924/tools/bin/../lib/gcc/arm-none-eabi/7.3.1/../../../../arm-none-eabi/lib/thumb/v7e-m/fpv4-sp/hard/crt0.o
LOAD Core/Src/GFX_BW.o
LOAD Core/Src/SSD1306_OLED.o
LOAD Core/Src/bmp280.o
LOAD Core/Src/freertos.o
LOAD Core/Src/gpio.o
LOAD Core/Src/i2c.o
LOAD Core/Src/main.o
LOAD Core/Src/printf.o
LOAD Core/Src/stm32f4xx_hal_msp.o
LOAD Core/Src/stm32f4xx_hal_timebase_tim.o
LOAD Core/Src/stm32f4xx_it.o
LOAD Core/Src/syscalls.o
LOAD Core/Src/sysmem.o
LOAD Core/Src/system_stm32f4xx.o
LOAD Core/Src/usart.o
LOAD Core/Startup/startup_stm32f411retx.o
LOAD Drivers/STM32F4xx_HAL_Driver/Src/stm32f4xx_hal.o
LOAD Drivers/STM32F4xx_HAL_Driver/Src/stm32f4xx_hal_cortex.o
LOAD Drivers/STM32F4xx_HAL_Driver/Src/stm32f4xx_hal_dma.o
LOAD Drivers/STM32F4xx_HAL_Driver/Src/stm32f4xx_hal_dma_ex.o
LOAD Drivers/STM32F4xx_HAL_Driver/Src/stm32f4xx_hal_exti.o
LOAD Drivers/STM32F4xx_HAL_Driver/Src/stm32f4xx_hal_flash.o
LOAD Drivers/STM32F4xx_HAL_Driver/Src/stm32f4xx_hal_flash_ex.o
LOAD Drivers/STM32F4xx_HAL_Driver/Src/stm32f4xx_hal_flash_ramfunc.o
LOAD Drivers/STM32F4xx_HAL_Driver/Src/stm32f4xx_hal_gpio.o
LOAD Drivers/STM32F4xx_HAL_Driver/Src/stm32f4xx_hal_i2c.o
LOAD Drivers/STM32F4xx_HAL_Driver/Src/stm32f4xx_hal_i2c_ex.o
LOAD Drivers/STM32F4xx_HAL_Driver/Src/stm32f4xx_hal_pwr.o
LOAD Drivers/STM32F4xx_HAL_Driver/Src/stm32f4xx_hal_pwr_ex.o
LOAD Drivers/STM32F4xx_HAL_Driver/Src/stm32f4xx_hal_rcc.o
LOAD Drivers/STM32F4xx_HAL_Driver/Src/stm32f4xx_hal_rcc_ex.o
LOAD Drivers/STM32F4xx_HAL_Driver/Src/stm32f4xx_hal_tim.o
LOAD Drivers/STM32F4xx_HAL_Driver/Src/stm32f4xx_hal_tim_ex.o
LOAD Drivers/STM32F4xx_HAL_Driver/Src/stm32f4xx_hal_uart.o
LOAD Middlewares/Third_Party/FreeRTOS/Source/CMSIS_RTOS_V2/cmsis_os2.o
LOAD Middlewares/Third_Party/FreeRTOS/Source/croutine.o
LOAD Middlewares/Third_Party/FreeRTOS/Source/event_groups.o
LOAD Middlewares/Third_Party/FreeRTOS/Source/list.o
LOAD Middlewares/Third_Party/FreeRTOS/Source/queue.o
LOAD Middlewares/Third_Party/FreeRTOS/Source/stream_buffer.o
LOAD Middlewares/Third_Party/FreeRTOS/Source/tasks.o
LOAD Middlewares/Third_Party/FreeRTOS/Source/timers.o
LOAD Middlewares/Third_Party/FreeRTOS/Source/portable/GCC/ARM_CM4F/port.o
LOAD Middlewares/Third_Party/FreeRTOS/Source/portable/MemMang/heap_4.o
START GROUP
LOAD d:/stm32cubeide_1.5.0/stm32cubeide/plugins/com.st.stm32cube.ide.mcu.externaltools.gnu-tools-for-stm32.7-2018-q2-update.win32_1.5.0.202011040924/tools/bin/../lib/gcc/arm-none-eabi/7.3.1/../../../../arm-none-eabi/lib/thumb/v7e-m/fpv4-sp/hard\libc_nano.a
LOAD d:/stm32cubeide_1.5.0/stm32cubeide/plugins/com.st.stm32cube.ide.mcu.externaltools.gnu-tools-for-stm32.7-2018-q2-update.win32_1.5.0.202011040924/tools/bin/../lib/gcc/arm-none-eabi/7.3.1/../../../../arm-none-eabi/lib/thumb/v7e-m/fpv4-sp/hard\libm.a
END GROUP
START GROUP
LOAD d:/stm32cubeide_1.5.0/stm32cubeide/plugins/com.st.stm32cube.ide.mcu.externaltools.gnu-tools-for-stm32.7-2018-q2-update.win32_1.5.0.202011040924/tools/bin/../lib/gcc/arm-none-eabi/7.3.1/thumb/v7e-m/fpv4-sp/hard\libgcc.a
LOAD d:/stm32cubeide_1.5.0/stm32cubeide/plugins/com.st.stm32cube.ide.mcu.externaltools.gnu-tools-for-stm32.7-2018-q2-update.win32_1.5.0.202011040924/tools/bin/../lib/gcc/arm-none-eabi/7.3.1/../../../../arm-none-eabi/lib/thumb/v7e-m/fpv4-sp/hard\libc_nano.a
END GROUP
START GROUP
LOAD d:/stm32cubeide_1.5.0/stm32cubeide/plugins/com.st.stm32cube.ide.mcu.externaltools.gnu-tools-for-stm32.7-2018-q2-update.win32_1.5.0.202011040924/tools/bin/../lib/gcc/arm-none-eabi/7.3.1/thumb/v7e-m/fpv4-sp/hard\libgcc.a
LOAD d:/stm32cubeide_1.5.0/stm32cubeide/plugins/com.st.stm32cube.ide.mcu.externaltools.gnu-tools-for-stm32.7-2018-q2-update.win32_1.5.0.202011040924/tools/bin/../lib/gcc/arm-none-eabi/7.3.1/../../../../arm-none-eabi/lib/thumb/v7e-m/fpv4-sp/hard\libc_nano.a
LOAD d:/stm32cubeide_1.5.0/stm32cubeide/plugins/com.st.stm32cube.ide.mcu.externaltools.gnu-tools-for-stm32.7-2018-q2-update.win32_1.5.0.202011040924/tools/bin/../lib/gcc/arm-none-eabi/7.3.1/../../../../arm-none-eabi/lib/thumb/v7e-m/fpv4-sp/hard\libnosys.a
END GROUP
START GROUP
LOAD d:/stm32cubeide_1.5.0/stm32cubeide/plugins/com.st.stm32cube.ide.mcu.externaltools.gnu-tools-for-stm32.7-2018-q2-update.win32_1.5.0.202011040924/tools/bin/../lib/gcc/arm-none-eabi/7.3.1/thumb/v7e-m/fpv4-sp/hard\libgcc.a
LOAD d:/stm32cubeide_1.5.0/stm32cubeide/plugins/com.st.stm32cube.ide.mcu.externaltools.gnu-tools-for-stm32.7-2018-q2-update.win32_1.5.0.202011040924/tools/bin/../lib/gcc/arm-none-eabi/7.3.1/../../../../arm-none-eabi/lib/thumb/v7e-m/fpv4-sp/hard\libc_nano.a
LOAD d:/stm32cubeide_1.5.0/stm32cubeide/plugins/com.st.stm32cube.ide.mcu.externaltools.gnu-tools-for-stm32.7-2018-q2-update.win32_1.5.0.202011040924/tools/bin/../lib/gcc/arm-none-eabi/7.3.1/../../../../arm-none-eabi/lib/thumb/v7e-m/fpv4-sp/hard\libnosys.a
END GROUP
LOAD d:/stm32cubeide_1.5.0/stm32cubeide/plugins/com.st.stm32cube.ide.mcu.externaltools.gnu-tools-for-stm32.7-2018-q2-update.win32_1.5.0.202011040924/tools/bin/../lib/gcc/arm-none-eabi/7.3.1/thumb/v7e-m/fpv4-sp/hard/crtend.o
LOAD d:/stm32cubeide_1.5.0/stm32cubeide/plugins/com.st.stm32cube.ide.mcu.externaltools.gnu-tools-for-stm32.7-2018-q2-update.win32_1.5.0.202011040924/tools/bin/../lib/gcc/arm-none-eabi/7.3.1/thumb/v7e-m/fpv4-sp/hard/crtn.o
                0x0000000020020000                _estack = (ORIGIN (RAM) + LENGTH (RAM))
                0x0000000000000200                _Min_Heap_Size = 0x200
                0x0000000000000400                _Min_Stack_Size = 0x400

.isr_vector     0x0000000008000000      0x198
                0x0000000008000000                . = ALIGN (0x4)
 *(.isr_vector)
 .isr_vector    0x0000000008000000      0x198 Core/Startup/startup_stm32f411retx.o
                0x0000000008000000                g_pfnVectors
                0x0000000008000198                . = ALIGN (0x4)

.text           0x00000000080001a0     0xa704
                0x00000000080001a0                . = ALIGN (0x4)
 *(.text)
 .text          0x00000000080001a0       0x40 d:/stm32cubeide_1.5.0/stm32cubeide/plugins/com.st.stm32cube.ide.mcu.externaltools.gnu-tools-for-stm32.7-2018-q2-update.win32_1.5.0.202011040924/tools/bin/../lib/gcc/arm-none-eabi/7.3.1/thumb/v7e-m/fpv4-sp/hard/crtbegin.o
 .text          0x00000000080001e0      0x378 d:/stm32cubeide_1.5.0/stm32cubeide/plugins/com.st.stm32cube.ide.mcu.externaltools.gnu-tools-for-stm32.7-2018-q2-update.win32_1.5.0.202011040924/tools/bin/../lib/gcc/arm-none-eabi/7.3.1/thumb/v7e-m/fpv4-sp/hard\libgcc.a(_arm_addsubdf3.o)
                0x00000000080001e0                __aeabi_drsub
                0x00000000080001e8                __aeabi_dsub
                0x00000000080001e8                __subdf3
                0x00000000080001ec                __aeabi_dadd
                0x00000000080001ec                __adddf3
                0x0000000008000464                __floatunsidf
                0x0000000008000464                __aeabi_ui2d
                0x0000000008000484                __floatsidf
                0x0000000008000484                __aeabi_i2d
                0x00000000080004a8                __aeabi_f2d
                0x00000000080004a8                __extendsfdf2
                0x00000000080004ec                __floatundidf
                0x00000000080004ec                __aeabi_ul2d
                0x00000000080004fc                __floatdidf
                0x00000000080004fc                __aeabi_l2d
 .text          0x0000000008000558      0x424 d:/stm32cubeide_1.5.0/stm32cubeide/plugins/com.st.stm32cube.ide.mcu.externaltools.gnu-tools-for-stm32.7-2018-q2-update.win32_1.5.0.202011040924/tools/bin/../lib/gcc/arm-none-eabi/7.3.1/thumb/v7e-m/fpv4-sp/hard\libgcc.a(_arm_muldivdf3.o)
                0x0000000008000558                __aeabi_dmul
                0x0000000008000558                __muldf3
                0x00000000080007ac                __divdf3
                0x00000000080007ac                __aeabi_ddiv
 .text          0x000000000800097c      0x110 d:/stm32cubeide_1.5.0/stm32cubeide/plugins/com.st.stm32cube.ide.mcu.externaltools.gnu-tools-for-stm32.7-2018-q2-update.win32_1.5.0.202011040924/tools/bin/../lib/gcc/arm-none-eabi/7.3.1/thumb/v7e-m/fpv4-sp/hard\libgcc.a(_arm_cmpdf2.o)
                0x000000000800097c                __gtdf2
                0x000000000800097c                __gedf2
                0x0000000008000984                __ltdf2
                0x0000000008000984                __ledf2
                0x000000000800098c                __nedf2
                0x000000000800098c                __eqdf2
                0x000000000800098c                __cmpdf2
                0x0000000008000a08                __aeabi_cdrcmple
                0x0000000008000a18                __aeabi_cdcmpeq
                0x0000000008000a18                __aeabi_cdcmple
                0x0000000008000a28                __aeabi_dcmpeq
                0x0000000008000a3c                __aeabi_dcmplt
                0x0000000008000a50                __aeabi_dcmple
                0x0000000008000a64                __aeabi_dcmpge
                0x0000000008000a78                __aeabi_dcmpgt
 .text          0x0000000008000a8c       0x50 d:/stm32cubeide_1.5.0/stm32cubeide/plugins/com.st.stm32cube.ide.mcu.externaltools.gnu-tools-for-stm32.7-2018-q2-update.win32_1.5.0.202011040924/tools/bin/../lib/gcc/arm-none-eabi/7.3.1/thumb/v7e-m/fpv4-sp/hard\libgcc.a(_arm_fixdfsi.o)
                0x0000000008000a8c                __aeabi_d2iz
                0x0000000008000a8c                __fixdfsi
 .text          0x0000000008000adc       0x40 d:/stm32cubeide_1.5.0/stm32cubeide/plugins/com.st.stm32cube.ide.mcu.externaltools.gnu-tools-for-stm32.7-2018-q2-update.win32_1.5.0.202011040924/tools/bin/../lib/gcc/arm-none-eabi/7.3.1/thumb/v7e-m/fpv4-sp/hard\libgcc.a(_arm_fixunsdfsi.o)
                0x0000000008000adc                __aeabi_d2uiz
                0x0000000008000adc                __fixunsdfsi
 .text          0x0000000008000b1c       0xa0 d:/stm32cubeide_1.5.0/stm32cubeide/plugins/com.st.stm32cube.ide.mcu.externaltools.gnu-tools-for-stm32.7-2018-q2-update.win32_1.5.0.202011040924/tools/bin/../lib/gcc/arm-none-eabi/7.3.1/thumb/v7e-m/fpv4-sp/hard\libgcc.a(_arm_truncdfsf2.o)
                0x0000000008000b1c                __truncdfsf2
                0x0000000008000b1c                __aeabi_d2f
 .text          0x0000000008000bbc       0x30 d:/stm32cubeide_1.5.0/stm32cubeide/plugins/com.st.stm32cube.ide.mcu.externaltools.gnu-tools-for-stm32.7-2018-q2-update.win32_1.5.0.202011040924/tools/bin/../lib/gcc/arm-none-eabi/7.3.1/thumb/v7e-m/fpv4-sp/hard\libgcc.a(_aeabi_uldivmod.o)
                0x0000000008000bbc                __aeabi_uldivmod
 .text          0x0000000008000bec      0x2cc d:/stm32cubeide_1.5.0/stm32cubeide/plugins/com.st.stm32cube.ide.mcu.externaltools.gnu-tools-for-stm32.7-2018-q2-update.win32_1.5.0.202011040924/tools/bin/../lib/gcc/arm-none-eabi/7.3.1/thumb/v7e-m/fpv4-sp/hard\libgcc.a(_udivmoddi4.o)
                0x0000000008000bec                __udivmoddi4
 .text          0x0000000008000eb8        0x4 d:/stm32cubeide_1.5.0/stm32cubeide/plugins/com.st.stm32cube.ide.mcu.externaltools.gnu-tools-for-stm32.7-2018-q2-update.win32_1.5.0.202011040924/tools/bin/../lib/gcc/arm-none-eabi/7.3.1/thumb/v7e-m/fpv4-sp/hard\libgcc.a(_dvmd_tls.o)
                0x0000000008000eb8                __aeabi_idiv0
                0x0000000008000eb8                __aeabi_ldiv0
 *(.text*)
 .text.GFX_SetFont
                0x0000000008000ebc       0x20 Core/Src/GFX_BW.o
                0x0000000008000ebc                GFX_SetFont
 .text.GFX_DrawChar
                0x0000000008000edc      0x174 Core/Src/GFX_BW.o
                0x0000000008000edc                GFX_DrawChar
 .text.GFX_DrawString
                0x0000000008001050       0xb4 Core/Src/GFX_BW.o
                0x0000000008001050                GFX_DrawString
 .text.GFX_WriteLine
                0x0000000008001104      0x11c Core/Src/GFX_BW.o
                0x0000000008001104                GFX_WriteLine
 .text.GFX_DrawFastVLine
                0x0000000008001220       0x2e Core/Src/GFX_BW.o
                0x0000000008001220                GFX_DrawFastVLine
 .text.GFX_DrawFillRectangle
                0x000000000800124e       0x44 Core/Src/GFX_BW.o
                0x000000000800124e                GFX_DrawFillRectangle
 *fill*         0x0000000008001292        0x2 
 .text.SSD1306_Command
                0x0000000008001294       0x34 Core/Src/SSD1306_OLED.o
                0x0000000008001294                SSD1306_Command
 .text.SSD1306_Data
                0x00000000080012c8       0x34 Core/Src/SSD1306_OLED.o
                0x00000000080012c8                SSD1306_Data
 .text.SSD1306_DrawPixel
                0x00000000080012fc      0x120 Core/Src/SSD1306_OLED.o
                0x00000000080012fc                SSD1306_DrawPixel
 .text.SSD1306_Clear
                0x000000000800141c       0x40 Core/Src/SSD1306_OLED.o
                0x000000000800141c                SSD1306_Clear
 .text.SSD1306_Display
                0x000000000800145c       0x3c Core/Src/SSD1306_OLED.o
                0x000000000800145c                SSD1306_Display
 .text.SSD1306_Init
                0x0000000008001498       0xb0 Core/Src/SSD1306_OLED.o
                0x0000000008001498                SSD1306_Init
 .text.Read8    0x0000000008001548       0x3e Core/Src/bmp280.o
                0x0000000008001548                Read8
 .text.Write8   0x0000000008001586       0x3e Core/Src/bmp280.o
                0x0000000008001586                Write8
 .text.Read16   0x00000000080015c4       0x4c Core/Src/bmp280.o
                0x00000000080015c4                Read16
 .text.Read24   0x0000000008001610       0x4a Core/Src/bmp280.o
                0x0000000008001610                Read24
 .text.BMP280_SetMode
                0x000000000800165a       0x52 Core/Src/bmp280.o
                0x000000000800165a                BMP280_SetMode
 .text.BMP280_SetPressureOversampling
                0x00000000080016ac       0x54 Core/Src/bmp280.o
                0x00000000080016ac                BMP280_SetPressureOversampling
 .text.BMP280_SetTemperatureOversampling
                0x0000000008001700       0x4e Core/Src/bmp280.o
                0x0000000008001700                BMP280_SetTemperatureOversampling
 .text.BMP280_ReadTemperatureRaw
                0x000000000800174e       0x24 Core/Src/bmp280.o
                0x000000000800174e                BMP280_ReadTemperatureRaw
 .text.BMP280_ReadPressureRaw
                0x0000000008001772       0x24 Core/Src/bmp280.o
                0x0000000008001772                BMP280_ReadPressureRaw
 *fill*         0x0000000008001796        0x2 
 .text.BMP280_ReadTemperature
                0x0000000008001798       0x9c Core/Src/bmp280.o
                0x0000000008001798                BMP280_ReadTemperature
 .text.BMP280_ReadPressureAndTemperature
                0x0000000008001834      0x16c Core/Src/bmp280.o
                0x0000000008001834                BMP280_ReadPressureAndTemperature
 .text.BMP280_Init
                0x00000000080019a0      0x112 Core/Src/bmp280.o
                0x00000000080019a0                BMP280_Init
 *fill*         0x0000000008001ab2        0x2 
 .text._putchar
                0x0000000008001ab4       0x40 Core/Src/freertos.o
                0x0000000008001ab4                _putchar
 .text.MX_FREERTOS_Init
                0x0000000008001af4       0xe8 Core/Src/freertos.o
                0x0000000008001af4                MX_FREERTOS_Init
 .text.StartHeartbeatTask
                0x0000000008001bdc       0x20 Core/Src/freertos.o
                0x0000000008001bdc                StartHeartbeatTask
 .text.StartBmp280Task
                0x0000000008001bfc       0xd0 Core/Src/freertos.o
                0x0000000008001bfc                StartBmp280Task
 .text.StartOledTask
                0x0000000008001ccc      0x128 Core/Src/freertos.o
                0x0000000008001ccc                StartOledTask
 .text.TimerBmpDataCallback
                0x0000000008001df4       0x20 Core/Src/freertos.o
                0x0000000008001df4                TimerBmpDataCallback
 .text.MX_GPIO_Init
                0x0000000008001e14       0xe0 Core/Src/gpio.o
                0x0000000008001e14                MX_GPIO_Init
 .text.MX_I2C1_Init
                0x0000000008001ef4       0x5c Core/Src/i2c.o
                0x0000000008001ef4                MX_I2C1_Init
 .text.HAL_I2C_MspInit
                0x0000000008001f50       0x90 Core/Src/i2c.o
                0x0000000008001f50                HAL_I2C_MspInit
 .text.main     0x0000000008001fe0       0x26 Core/Src/main.o
                0x0000000008001fe0                main
 *fill*         0x0000000008002006        0x2 
 .text.SystemClock_Config
                0x0000000008002008       0xd4 Core/Src/main.o
                0x0000000008002008                SystemClock_Config
 .text.HAL_TIM_PeriodElapsedCallback
                0x00000000080020dc       0x24 Core/Src/main.o
                0x00000000080020dc                HAL_TIM_PeriodElapsedCallback
 .text.Error_Handler
                0x0000000008002100        0x8 Core/Src/main.o
                0x0000000008002100                Error_Handler
 .text._out_buffer
                0x0000000008002108       0x2e Core/Src/printf.o
 .text._out_null
                0x0000000008002136       0x1c Core/Src/printf.o
 .text._out_char
                0x0000000008002152       0x26 Core/Src/printf.o
 .text._strnlen_s
                0x0000000008002178       0x3a Core/Src/printf.o
 .text._is_digit
                0x00000000080021b2       0x2e Core/Src/printf.o
 .text._atoi    0x00000000080021e0       0x48 Core/Src/printf.o
 .text._out_rev
                0x0000000008002228       0xa0 Core/Src/printf.o
 .text._ntoa_format
                0x00000000080022c8      0x1b8 Core/Src/printf.o
 .text._ntoa_long
                0x0000000008002480       0xce Core/Src/printf.o
 .text._ntoa_long_long
                0x000000000800254e       0xde Core/Src/printf.o
 *fill*         0x000000000800262c        0x4 
 .text._ftoa    0x0000000008002630      0x4d4 Core/Src/printf.o
 *fill*         0x0000000008002b04        0x4 
 .text._etoa    0x0000000008002b08      0x530 Core/Src/printf.o
 .text._vsnprintf
                0x0000000008003038      0x96c Core/Src/printf.o
 .text.printf_  0x00000000080039a4       0x38 Core/Src/printf.o
                0x00000000080039a4                printf_
 .text.sprintf_
                0x00000000080039dc       0x38 Core/Src/printf.o
                0x00000000080039dc                sprintf_
 .text.HAL_MspInit
                0x0000000008003a14       0x58 Core/Src/stm32f4xx_hal_msp.o
                0x0000000008003a14                HAL_MspInit
 .text.HAL_InitTick
                0x0000000008003a6c       0xb0 Core/Src/stm32f4xx_hal_timebase_tim.o
                0x0000000008003a6c                HAL_InitTick
 .text.NMI_Handler
                0x0000000008003b1c        0x6 Core/Src/stm32f4xx_it.o
                0x0000000008003b1c                NMI_Handler
 .text.HardFault_Handler
                0x0000000008003b22        0x6 Core/Src/stm32f4xx_it.o
                0x0000000008003b22                HardFault_Handler
 .text.MemManage_Handler
                0x0000000008003b28        0x6 Core/Src/stm32f4xx_it.o
                0x0000000008003b28                MemManage_Handler
 .text.BusFault_Handler
                0x0000000008003b2e        0x6 Core/Src/stm32f4xx_it.o
                0x0000000008003b2e                BusFault_Handler
 .text.UsageFault_Handler
                0x0000000008003b34        0x6 Core/Src/stm32f4xx_it.o
                0x0000000008003b34                UsageFault_Handler
 .text.DebugMon_Handler
                0x0000000008003b3a        0xe Core/Src/stm32f4xx_it.o
                0x0000000008003b3a                DebugMon_Handler
 .text.TIM1_UP_TIM10_IRQHandler
                0x0000000008003b48       0x14 Core/Src/stm32f4xx_it.o
                0x0000000008003b48                TIM1_UP_TIM10_IRQHandler
 .text.SystemInit
                0x0000000008003b5c       0x2c Core/Src/system_stm32f4xx.o
                0x0000000008003b5c                SystemInit
 .text.MX_USART2_UART_Init
                0x0000000008003b88       0x54 Core/Src/usart.o
                0x0000000008003b88                MX_USART2_UART_Init
 .text.HAL_UART_MspInit
                0x0000000008003bdc       0x90 Core/Src/usart.o
                0x0000000008003bdc                HAL_UART_MspInit
 .text.Reset_Handler
                0x0000000008003c6c       0x50 Core/Startup/startup_stm32f411retx.o
                0x0000000008003c6c                Reset_Handler
 .text.Default_Handler
                0x0000000008003cbc        0x2 Core/Startup/startup_stm32f411retx.o
                0x0000000008003cbc                RTC_Alarm_IRQHandler
                0x0000000008003cbc                EXTI2_IRQHandler
                0x0000000008003cbc                SPI4_IRQHandler
                0x0000000008003cbc                TIM1_CC_IRQHandler
                0x0000000008003cbc                DMA2_Stream5_IRQHandler
                0x0000000008003cbc                DMA1_Stream5_IRQHandler
                0x0000000008003cbc                PVD_IRQHandler
                0x0000000008003cbc                SDIO_IRQHandler
                0x0000000008003cbc                TAMP_STAMP_IRQHandler
                0x0000000008003cbc                EXTI3_IRQHandler
                0x0000000008003cbc                I2C3_ER_IRQHandler
                0x0000000008003cbc                EXTI0_IRQHandler
                0x0000000008003cbc                I2C2_EV_IRQHandler
                0x0000000008003cbc                DMA1_Stream2_IRQHandler
                0x0000000008003cbc                FPU_IRQHandler
                0x0000000008003cbc                DMA2_Stream2_IRQHandler
                0x0000000008003cbc                SPI1_IRQHandler
                0x0000000008003cbc                TIM1_BRK_TIM9_IRQHandler
                0x0000000008003cbc                DMA2_Stream3_IRQHandler
                0x0000000008003cbc                USART6_IRQHandler
                0x0000000008003cbc                DMA2_Stream0_IRQHandler
                0x0000000008003cbc                TIM4_IRQHandler
                0x0000000008003cbc                I2C1_EV_IRQHandler
                0x0000000008003cbc                DMA1_Stream6_IRQHandler
                0x0000000008003cbc                DMA1_Stream1_IRQHandler
                0x0000000008003cbc                TIM3_IRQHandler
                0x0000000008003cbc                RCC_IRQHandler
                0x0000000008003cbc                Default_Handler
                0x0000000008003cbc                EXTI15_10_IRQHandler
                0x0000000008003cbc                ADC_IRQHandler
                0x0000000008003cbc                DMA1_Stream7_IRQHandler
                0x0000000008003cbc                SPI5_IRQHandler
                0x0000000008003cbc                TIM5_IRQHandler
                0x0000000008003cbc                DMA2_Stream7_IRQHandler
                0x0000000008003cbc                I2C3_EV_IRQHandler
                0x0000000008003cbc                EXTI9_5_IRQHandler
                0x0000000008003cbc                RTC_WKUP_IRQHandler
                0x0000000008003cbc                SPI2_IRQHandler
                0x0000000008003cbc                DMA1_Stream0_IRQHandler
                0x0000000008003cbc                EXTI4_IRQHandler
                0x0000000008003cbc                WWDG_IRQHandler
                0x0000000008003cbc                TIM2_IRQHandler
                0x0000000008003cbc                OTG_FS_WKUP_IRQHandler
                0x0000000008003cbc                TIM1_TRG_COM_TIM11_IRQHandler
                0x0000000008003cbc                EXTI1_IRQHandler
                0x0000000008003cbc                USART2_IRQHandler
                0x0000000008003cbc                I2C2_ER_IRQHandler
                0x0000000008003cbc                DMA2_Stream1_IRQHandler
                0x0000000008003cbc                FLASH_IRQHandler
                0x0000000008003cbc                DMA2_Stream4_IRQHandler
                0x0000000008003cbc                USART1_IRQHandler
                0x0000000008003cbc                OTG_FS_IRQHandler
                0x0000000008003cbc                SPI3_IRQHandler
                0x0000000008003cbc                DMA1_Stream4_IRQHandler
                0x0000000008003cbc                I2C1_ER_IRQHandler
                0x0000000008003cbc                DMA2_Stream6_IRQHandler
                0x0000000008003cbc                DMA1_Stream3_IRQHandler
 *fill*         0x0000000008003cbe        0x2 
 .text.HAL_Init
                0x0000000008003cc0       0x44 Drivers/STM32F4xx_HAL_Driver/Src/stm32f4xx_hal.o
                0x0000000008003cc0                HAL_Init
 .text.HAL_IncTick
                0x0000000008003d04       0x28 Drivers/STM32F4xx_HAL_Driver/Src/stm32f4xx_hal.o
                0x0000000008003d04                HAL_IncTick
 .text.HAL_GetTick
                0x0000000008003d2c       0x18 Drivers/STM32F4xx_HAL_Driver/Src/stm32f4xx_hal.o
                0x0000000008003d2c                HAL_GetTick
 .text.__NVIC_SetPriorityGrouping
                0x0000000008003d44       0x48 Drivers/STM32F4xx_HAL_Driver/Src/stm32f4xx_hal_cortex.o
 .text.__NVIC_GetPriorityGrouping
                0x0000000008003d8c       0x1c Drivers/STM32F4xx_HAL_Driver/Src/stm32f4xx_hal_cortex.o
 .text.__NVIC_EnableIRQ
                0x0000000008003da8       0x3c Drivers/STM32F4xx_HAL_Driver/Src/stm32f4xx_hal_cortex.o
 .text.__NVIC_SetPriority
                0x0000000008003de4       0x54 Drivers/STM32F4xx_HAL_Driver/Src/stm32f4xx_hal_cortex.o
 .text.NVIC_EncodePriority
                0x0000000008003e38       0x66 Drivers/STM32F4xx_HAL_Driver/Src/stm32f4xx_hal_cortex.o
 .text.HAL_NVIC_SetPriorityGrouping
                0x0000000008003e9e       0x16 Drivers/STM32F4xx_HAL_Driver/Src/stm32f4xx_hal_cortex.o
                0x0000000008003e9e                HAL_NVIC_SetPriorityGrouping
 .text.HAL_NVIC_SetPriority
                0x0000000008003eb4       0x38 Drivers/STM32F4xx_HAL_Driver/Src/stm32f4xx_hal_cortex.o
                0x0000000008003eb4                HAL_NVIC_SetPriority
 .text.HAL_NVIC_EnableIRQ
                0x0000000008003eec       0x1c Drivers/STM32F4xx_HAL_Driver/Src/stm32f4xx_hal_cortex.o
                0x0000000008003eec                HAL_NVIC_EnableIRQ
 .text.HAL_GPIO_Init
                0x0000000008003f08      0x304 Drivers/STM32F4xx_HAL_Driver/Src/stm32f4xx_hal_gpio.o
                0x0000000008003f08                HAL_GPIO_Init
 .text.HAL_GPIO_WritePin
                0x000000000800420c       0x32 Drivers/STM32F4xx_HAL_Driver/Src/stm32f4xx_hal_gpio.o
                0x000000000800420c                HAL_GPIO_WritePin
 .text.HAL_GPIO_TogglePin
                0x000000000800423e       0x36 Drivers/STM32F4xx_HAL_Driver/Src/stm32f4xx_hal_gpio.o
                0x000000000800423e                HAL_GPIO_TogglePin
 .text.HAL_I2C_Init
                0x0000000008004274      0x270 Drivers/STM32F4xx_HAL_Driver/Src/stm32f4xx_hal_i2c.o
                0x0000000008004274                HAL_I2C_Init
 .text.HAL_I2C_Mem_Write
                0x00000000080044e4      0x1f4 Drivers/STM32F4xx_HAL_Driver/Src/stm32f4xx_hal_i2c.o
                0x00000000080044e4                HAL_I2C_Mem_Write
 .text.HAL_I2C_Mem_Read
                0x00000000080046d8      0x44c Drivers/STM32F4xx_HAL_Driver/Src/stm32f4xx_hal_i2c.o
                0x00000000080046d8                HAL_I2C_Mem_Read
 .text.I2C_RequestMemoryWrite
                0x0000000008004b24      0x12c Drivers/STM32F4xx_HAL_Driver/Src/stm32f4xx_hal_i2c.o
 .text.I2C_RequestMemoryRead
                0x0000000008004c50      0x1d0 Drivers/STM32F4xx_HAL_Driver/Src/stm32f4xx_hal_i2c.o
 .text.I2C_WaitOnFlagUntilTimeout
                0x0000000008004e20       0xae Drivers/STM32F4xx_HAL_Driver/Src/stm32f4xx_hal_i2c.o
 .text.I2C_WaitOnMasterAddressFlagUntilTimeout
                0x0000000008004ece       0xfe Drivers/STM32F4xx_HAL_Driver/Src/stm32f4xx_hal_i2c.o
 .text.I2C_WaitOnTXEFlagUntilTimeout
                0x0000000008004fcc       0x82 Drivers/STM32F4xx_HAL_Driver/Src/stm32f4xx_hal_i2c.o
 .text.I2C_WaitOnBTFFlagUntilTimeout
                0x000000000800504e       0x82 Drivers/STM32F4xx_HAL_Driver/Src/stm32f4xx_hal_i2c.o
 .text.I2C_WaitOnRXNEFlagUntilTimeout
                0x00000000080050d0       0xac Drivers/STM32F4xx_HAL_Driver/Src/stm32f4xx_hal_i2c.o
 .text.I2C_IsAcknowledgeFailed
                0x000000000800517c       0x5e Drivers/STM32F4xx_HAL_Driver/Src/stm32f4xx_hal_i2c.o
 *fill*         0x00000000080051da        0x2 
 .text.HAL_RCC_OscConfig
                0x00000000080051dc      0x4e0 Drivers/STM32F4xx_HAL_Driver/Src/stm32f4xx_hal_rcc.o
                0x00000000080051dc                HAL_RCC_OscConfig
 .text.HAL_RCC_ClockConfig
                0x00000000080056bc      0x1cc Drivers/STM32F4xx_HAL_Driver/Src/stm32f4xx_hal_rcc.o
                0x00000000080056bc                HAL_RCC_ClockConfig
 .text.HAL_RCC_GetSysClockFreq
                0x0000000008005888      0x1b0 Drivers/STM32F4xx_HAL_Driver/Src/stm32f4xx_hal_rcc.o
                0x0000000008005888                HAL_RCC_GetSysClockFreq
 .text.HAL_RCC_GetHCLKFreq
                0x0000000008005a38       0x18 Drivers/STM32F4xx_HAL_Driver/Src/stm32f4xx_hal_rcc.o
                0x0000000008005a38                HAL_RCC_GetHCLKFreq
 .text.HAL_RCC_GetPCLK1Freq
                0x0000000008005a50       0x28 Drivers/STM32F4xx_HAL_Driver/Src/stm32f4xx_hal_rcc.o
                0x0000000008005a50                HAL_RCC_GetPCLK1Freq
 .text.HAL_RCC_GetPCLK2Freq
                0x0000000008005a78       0x28 Drivers/STM32F4xx_HAL_Driver/Src/stm32f4xx_hal_rcc.o
                0x0000000008005a78                HAL_RCC_GetPCLK2Freq
 .text.HAL_RCC_GetClockConfig
                0x0000000008005aa0       0x64 Drivers/STM32F4xx_HAL_Driver/Src/stm32f4xx_hal_rcc.o
                0x0000000008005aa0                HAL_RCC_GetClockConfig
 .text.HAL_TIM_Base_Init
                0x0000000008005b04       0x56 Drivers/STM32F4xx_HAL_Driver/Src/stm32f4xx_hal_tim.o
                0x0000000008005b04                HAL_TIM_Base_Init
 .text.HAL_TIM_Base_MspInit
                0x0000000008005b5a       0x14 Drivers/STM32F4xx_HAL_Driver/Src/stm32f4xx_hal_tim.o
                0x0000000008005b5a                HAL_TIM_Base_MspInit
 .text.HAL_TIM_Base_Start_IT
                0x0000000008005b6e       0x48 Drivers/STM32F4xx_HAL_Driver/Src/stm32f4xx_hal_tim.o
                0x0000000008005b6e                HAL_TIM_Base_Start_IT
 .text.HAL_TIM_IRQHandler
                0x0000000008005bb6      0x210 Drivers/STM32F4xx_HAL_Driver/Src/stm32f4xx_hal_tim.o
                0x0000000008005bb6                HAL_TIM_IRQHandler
 .text.HAL_TIM_OC_DelayElapsedCallback
                0x0000000008005dc6       0x14 Drivers/STM32F4xx_HAL_Driver/Src/stm32f4xx_hal_tim.o
                0x0000000008005dc6                HAL_TIM_OC_DelayElapsedCallback
 .text.HAL_TIM_IC_CaptureCallback
                0x0000000008005dda       0x14 Drivers/STM32F4xx_HAL_Driver/Src/stm32f4xx_hal_tim.o
                0x0000000008005dda                HAL_TIM_IC_CaptureCallback
 .text.HAL_TIM_PWM_PulseFinishedCallback
                0x0000000008005dee       0x14 Drivers/STM32F4xx_HAL_Driver/Src/stm32f4xx_hal_tim.o
                0x0000000008005dee                HAL_TIM_PWM_PulseFinishedCallback
 .text.HAL_TIM_TriggerCallback
                0x0000000008005e02       0x14 Drivers/STM32F4xx_HAL_Driver/Src/stm32f4xx_hal_tim.o
                0x0000000008005e02                HAL_TIM_TriggerCallback
 *fill*         0x0000000008005e16        0x2 
 .text.TIM_Base_SetConfig
                0x0000000008005e18      0x100 Drivers/STM32F4xx_HAL_Driver/Src/stm32f4xx_hal_tim.o
                0x0000000008005e18                TIM_Base_SetConfig
 .text.HAL_TIMEx_CommutCallback
                0x0000000008005f18       0x14 Drivers/STM32F4xx_HAL_Driver/Src/stm32f4xx_hal_tim_ex.o
                0x0000000008005f18                HAL_TIMEx_CommutCallback
 .text.HAL_TIMEx_BreakCallback
                0x0000000008005f2c       0x14 Drivers/STM32F4xx_HAL_Driver/Src/stm32f4xx_hal_tim_ex.o
                0x0000000008005f2c                HAL_TIMEx_BreakCallback
 .text.HAL_UART_Init
                0x0000000008005f40       0x9a Drivers/STM32F4xx_HAL_Driver/Src/stm32f4xx_hal_uart.o
                0x0000000008005f40                HAL_UART_Init
 .text.HAL_UART_Transmit
                0x0000000008005fda      0x132 Drivers/STM32F4xx_HAL_Driver/Src/stm32f4xx_hal_uart.o
                0x0000000008005fda                HAL_UART_Transmit
 .text.UART_WaitOnFlagUntilTimeout
                0x000000000800610c       0x94 Drivers/STM32F4xx_HAL_Driver/Src/stm32f4xx_hal_uart.o
 .text.UART_SetConfig
                0x00000000080061a0      0x6f8 Drivers/STM32F4xx_HAL_Driver/Src/stm32f4xx_hal_uart.o
 .text.SVC_Setup
                0x0000000008006898        0xe Middlewares/Third_Party/FreeRTOS/Source/CMSIS_RTOS_V2/cmsis_os2.o
 *fill*         0x00000000080068a6        0x2 
 .text.osKernelInitialize
                0x00000000080068a8       0x68 Middlewares/Third_Party/FreeRTOS/Source/CMSIS_RTOS_V2/cmsis_os2.o
                0x00000000080068a8                osKernelInitialize
 .text.osKernelStart
                0x0000000008006910       0x6c Middlewares/Third_Party/FreeRTOS/Source/CMSIS_RTOS_V2/cmsis_os2.o
                0x0000000008006910                osKernelStart
 .text.osThreadNew
                0x000000000800697c      0x14c Middlewares/Third_Party/FreeRTOS/Source/CMSIS_RTOS_V2/cmsis_os2.o
                0x000000000800697c                osThreadNew
 .text.osDelay  0x0000000008006ac8       0x5c Middlewares/Third_Party/FreeRTOS/Source/CMSIS_RTOS_V2/cmsis_os2.o
                0x0000000008006ac8                osDelay
 .text.TimerCallback
                0x0000000008006b24       0x2a Middlewares/Third_Party/FreeRTOS/Source/CMSIS_RTOS_V2/cmsis_os2.o
 *fill*         0x0000000008006b4e        0x2 
 .text.osTimerNew
                0x0000000008006b50      0x108 Middlewares/Third_Party/FreeRTOS/Source/CMSIS_RTOS_V2/cmsis_os2.o
                0x0000000008006b50                osTimerNew
 .text.osTimerStart
                0x0000000008006c58       0x80 Middlewares/Third_Party/FreeRTOS/Source/CMSIS_RTOS_V2/cmsis_os2.o
                0x0000000008006c58                osTimerStart
 .text.osMutexNew
                0x0000000008006cd8      0x134 Middlewares/Third_Party/FreeRTOS/Source/CMSIS_RTOS_V2/cmsis_os2.o
                0x0000000008006cd8                osMutexNew
 .text.osMutexAcquire
                0x0000000008006e0c       0xbc Middlewares/Third_Party/FreeRTOS/Source/CMSIS_RTOS_V2/cmsis_os2.o
                0x0000000008006e0c                osMutexAcquire
 .text.osMutexRelease
                0x0000000008006ec8       0xa0 Middlewares/Third_Party/FreeRTOS/Source/CMSIS_RTOS_V2/cmsis_os2.o
                0x0000000008006ec8                osMutexRelease
 .text.osSemaphoreNew
                0x0000000008006f68      0x13c Middlewares/Third_Party/FreeRTOS/Source/CMSIS_RTOS_V2/cmsis_os2.o
                0x0000000008006f68                osSemaphoreNew
 .text.osSemaphoreAcquire
                0x00000000080070a4       0xcc Middlewares/Third_Party/FreeRTOS/Source/CMSIS_RTOS_V2/cmsis_os2.o
                0x00000000080070a4                osSemaphoreAcquire
 .text.osSemaphoreRelease
                0x0000000008007170       0xb0 Middlewares/Third_Party/FreeRTOS/Source/CMSIS_RTOS_V2/cmsis_os2.o
                0x0000000008007170                osSemaphoreRelease
 .text.osMessageQueueNew
                0x0000000008007220      0x10c Middlewares/Third_Party/FreeRTOS/Source/CMSIS_RTOS_V2/cmsis_os2.o
                0x0000000008007220                osMessageQueueNew
 .text.osMessageQueuePut
                0x000000000800732c       0xe8 Middlewares/Third_Party/FreeRTOS/Source/CMSIS_RTOS_V2/cmsis_os2.o
                0x000000000800732c                osMessageQueuePut
 .text.osMessageQueueGet
                0x0000000008007414       0xe4 Middlewares/Third_Party/FreeRTOS/Source/CMSIS_RTOS_V2/cmsis_os2.o
                0x0000000008007414                osMessageQueueGet
 .text.vApplicationGetIdleTaskMemory
                0x00000000080074f8       0x34 Middlewares/Third_Party/FreeRTOS/Source/CMSIS_RTOS_V2/cmsis_os2.o
                0x00000000080074f8                vApplicationGetIdleTaskMemory
 .text.vApplicationGetTimerTaskMemory
                0x000000000800752c       0x34 Middlewares/Third_Party/FreeRTOS/Source/CMSIS_RTOS_V2/cmsis_os2.o
                0x000000000800752c                vApplicationGetTimerTaskMemory
 .text.vListInitialise
                0x0000000008007560       0x40 Middlewares/Third_Party/FreeRTOS/Source/list.o
                0x0000000008007560                vListInitialise
 .text.vListInitialiseItem
                0x00000000080075a0       0x1a Middlewares/Third_Party/FreeRTOS/Source/list.o
                0x00000000080075a0                vListInitialiseItem
 .text.vListInsertEnd
                0x00000000080075ba       0x48 Middlewares/Third_Party/FreeRTOS/Source/list.o
                0x00000000080075ba                vListInsertEnd
 .text.vListInsert
                0x0000000008007602       0x72 Middlewares/Third_Party/FreeRTOS/Source/list.o
                0x0000000008007602                vListInsert
 .text.uxListRemove
                0x0000000008007674       0x54 Middlewares/Third_Party/FreeRTOS/Source/list.o
                0x0000000008007674                uxListRemove
 .text.xQueueGenericReset
                0x00000000080076c8       0xd0 Middlewares/Third_Party/FreeRTOS/Source/queue.o
                0x00000000080076c8                xQueueGenericReset
 .text.xQueueGenericCreateStatic
                0x0000000008007798       0xe6 Middlewares/Third_Party/FreeRTOS/Source/queue.o
                0x0000000008007798                xQueueGenericCreateStatic
 .text.xQueueGenericCreate
                0x000000000800787e       0x7e Middlewares/Third_Party/FreeRTOS/Source/queue.o
                0x000000000800787e                xQueueGenericCreate
 .text.prvInitialiseNewQueue
                0x00000000080078fc       0x46 Middlewares/Third_Party/FreeRTOS/Source/queue.o
 .text.prvInitialiseMutex
                0x0000000008007942       0x34 Middlewares/Third_Party/FreeRTOS/Source/queue.o
 .text.xQueueCreateMutex
                0x0000000008007976       0x30 Middlewares/Third_Party/FreeRTOS/Source/queue.o
                0x0000000008007976                xQueueCreateMutex
 .text.xQueueCreateMutexStatic
                0x00000000080079a6       0x36 Middlewares/Third_Party/FreeRTOS/Source/queue.o
                0x00000000080079a6                xQueueCreateMutexStatic
 .text.xQueueGiveMutexRecursive
                0x00000000080079dc       0x66 Middlewares/Third_Party/FreeRTOS/Source/queue.o
                0x00000000080079dc                xQueueGiveMutexRecursive
 .text.xQueueTakeMutexRecursive
                0x0000000008007a42       0x6a Middlewares/Third_Party/FreeRTOS/Source/queue.o
                0x0000000008007a42                xQueueTakeMutexRecursive
 .text.xQueueCreateCountingSemaphoreStatic
                0x0000000008007aac       0x6a Middlewares/Third_Party/FreeRTOS/Source/queue.o
                0x0000000008007aac                xQueueCreateCountingSemaphoreStatic
 .text.xQueueCreateCountingSemaphore
                0x0000000008007b16       0x62 Middlewares/Third_Party/FreeRTOS/Source/queue.o
                0x0000000008007b16                xQueueCreateCountingSemaphore
 .text.xQueueGenericSend
                0x0000000008007b78      0x1f4 Middlewares/Third_Party/FreeRTOS/Source/queue.o
                0x0000000008007b78                xQueueGenericSend
 .text.xQueueGenericSendFromISR
                0x0000000008007d6c      0x128 Middlewares/Third_Party/FreeRTOS/Source/queue.o
                0x0000000008007d6c                xQueueGenericSendFromISR
 .text.xQueueGiveFromISR
                0x0000000008007e94      0x112 Middlewares/Third_Party/FreeRTOS/Source/queue.o
                0x0000000008007e94                xQueueGiveFromISR
 *fill*         0x0000000008007fa6        0x2 
 .text.xQueueReceive
                0x0000000008007fa8      0x1b8 Middlewares/Third_Party/FreeRTOS/Source/queue.o
                0x0000000008007fa8                xQueueReceive
 .text.xQueueSemaphoreTake
                0x0000000008008160      0x210 Middlewares/Third_Party/FreeRTOS/Source/queue.o
                0x0000000008008160                xQueueSemaphoreTake
 .text.xQueueReceiveFromISR
                0x0000000008008370       0xfa Middlewares/Third_Party/FreeRTOS/Source/queue.o
                0x0000000008008370                xQueueReceiveFromISR
 .text.vQueueDelete
                0x000000000800846a       0x44 Middlewares/Third_Party/FreeRTOS/Source/queue.o
                0x000000000800846a                vQueueDelete
 .text.prvGetDisinheritPriorityAfterTimeout
                0x00000000080084ae       0x30 Middlewares/Third_Party/FreeRTOS/Source/queue.o
 .text.prvCopyDataToQueue
                0x00000000080084de       0xd4 Middlewares/Third_Party/FreeRTOS/Source/queue.o
 .text.prvCopyDataFromQueue
                0x00000000080085b2       0x4c Middlewares/Third_Party/FreeRTOS/Source/queue.o
 .text.prvUnlockQueue
                0x00000000080085fe       0xa4 Middlewares/Third_Party/FreeRTOS/Source/queue.o
 .text.prvIsQueueEmpty
                0x00000000080086a2       0x2c Middlewares/Third_Party/FreeRTOS/Source/queue.o
 .text.prvIsQueueFull
                0x00000000080086ce       0x30 Middlewares/Third_Party/FreeRTOS/Source/queue.o
 *fill*         0x00000000080086fe        0x2 
 .text.vQueueAddToRegistry
                0x0000000008008700       0x50 Middlewares/Third_Party/FreeRTOS/Source/queue.o
                0x0000000008008700                vQueueAddToRegistry
 .text.vQueueUnregisterQueue
                0x0000000008008750       0x54 Middlewares/Third_Party/FreeRTOS/Source/queue.o
                0x0000000008008750                vQueueUnregisterQueue
 .text.vQueueWaitForMessageRestricted
                0x00000000080087a4       0x68 Middlewares/Third_Party/FreeRTOS/Source/queue.o
                0x00000000080087a4                vQueueWaitForMessageRestricted
 .text.xTaskCreateStatic
                0x000000000800880c       0xb4 Middlewares/Third_Party/FreeRTOS/Source/tasks.o
                0x000000000800880c                xTaskCreateStatic
 .text.xTaskCreate
                0x00000000080088c0       0x8a Middlewares/Third_Party/FreeRTOS/Source/tasks.o
                0x00000000080088c0                xTaskCreate
 .text.prvInitialiseNewTask
                0x000000000800894a      0x11c Middlewares/Third_Party/FreeRTOS/Source/tasks.o
 *fill*         0x0000000008008a66        0x2 
 .text.prvAddNewTaskToReadyList
                0x0000000008008a68       0xe0 Middlewares/Third_Party/FreeRTOS/Source/tasks.o
 .text.vTaskDelay
                0x0000000008008b48       0x68 Middlewares/Third_Party/FreeRTOS/Source/tasks.o
                0x0000000008008b48                vTaskDelay
 .text.vTaskStartScheduler
                0x0000000008008bb0       0xc8 Middlewares/Third_Party/FreeRTOS/Source/tasks.o
                0x0000000008008bb0                vTaskStartScheduler
 .text.vTaskSuspendAll
                0x0000000008008c78       0x1c Middlewares/Third_Party/FreeRTOS/Source/tasks.o
                0x0000000008008c78                vTaskSuspendAll
 .text.xTaskResumeAll
                0x0000000008008c94      0x138 Middlewares/Third_Party/FreeRTOS/Source/tasks.o
                0x0000000008008c94                xTaskResumeAll
 .text.xTaskGetTickCount
                0x0000000008008dcc       0x20 Middlewares/Third_Party/FreeRTOS/Source/tasks.o
                0x0000000008008dcc                xTaskGetTickCount
 .text.xTaskIncrementTick
                0x0000000008008dec      0x170 Middlewares/Third_Party/FreeRTOS/Source/tasks.o
                0x0000000008008dec                xTaskIncrementTick
 .text.vTaskSwitchContext
                0x0000000008008f5c       0xb8 Middlewares/Third_Party/FreeRTOS/Source/tasks.o
                0x0000000008008f5c                vTaskSwitchContext
 .text.vTaskPlaceOnEventList
                0x0000000008009014       0x48 Middlewares/Third_Party/FreeRTOS/Source/tasks.o
                0x0000000008009014                vTaskPlaceOnEventList
 .text.vTaskPlaceOnEventListRestricted
                0x000000000800905c       0x54 Middlewares/Third_Party/FreeRTOS/Source/tasks.o
                0x000000000800905c                vTaskPlaceOnEventListRestricted
 .text.xTaskRemoveFromEventList
                0x00000000080090b0       0xc4 Middlewares/Third_Party/FreeRTOS/Source/tasks.o
                0x00000000080090b0                xTaskRemoveFromEventList
 .text.vTaskInternalSetTimeOutState
                0x0000000008009174       0x2c Middlewares/Third_Party/FreeRTOS/Source/tasks.o
                0x0000000008009174                vTaskInternalSetTimeOutState
 .text.xTaskCheckForTimeOut
                0x00000000080091a0       0xc0 Middlewares/Third_Party/FreeRTOS/Source/tasks.o
                0x00000000080091a0                xTaskCheckForTimeOut
 .text.vTaskMissedYield
                0x0000000008009260       0x18 Middlewares/Third_Party/FreeRTOS/Source/tasks.o
                0x0000000008009260                vTaskMissedYield
 .text.prvIdleTask
                0x0000000008009278       0x30 Middlewares/Third_Party/FreeRTOS/Source/tasks.o
 .text.prvInitialiseTaskLists
                0x00000000080092a8       0x80 Middlewares/Third_Party/FreeRTOS/Source/tasks.o
 .text.prvCheckTasksWaitingTermination
                0x0000000008009328       0x58 Middlewares/Third_Party/FreeRTOS/Source/tasks.o
 .text.prvDeleteTCB
                0x0000000008009380       0x5c Middlewares/Third_Party/FreeRTOS/Source/tasks.o
 .text.prvResetNextTaskUnblockTime
                0x00000000080093dc       0x40 Middlewares/Third_Party/FreeRTOS/Source/tasks.o
 .text.xTaskGetCurrentTaskHandle
                0x000000000800941c       0x20 Middlewares/Third_Party/FreeRTOS/Source/tasks.o
                0x000000000800941c                xTaskGetCurrentTaskHandle
 .text.xTaskGetSchedulerState
                0x000000000800943c       0x3c Middlewares/Third_Party/FreeRTOS/Source/tasks.o
                0x000000000800943c                xTaskGetSchedulerState
 .text.xTaskPriorityInherit
                0x0000000008009478       0xd0 Middlewares/Third_Party/FreeRTOS/Source/tasks.o
                0x0000000008009478                xTaskPriorityInherit
 .text.xTaskPriorityDisinherit
                0x0000000008009548       0xd8 Middlewares/Third_Party/FreeRTOS/Source/tasks.o
                0x0000000008009548                xTaskPriorityDisinherit
 .text.vTaskPriorityDisinheritAfterTimeout
                0x0000000008009620      0x100 Middlewares/Third_Party/FreeRTOS/Source/tasks.o
                0x0000000008009620                vTaskPriorityDisinheritAfterTimeout
 .text.pvTaskIncrementMutexHeldCount
                0x0000000008009720       0x28 Middlewares/Third_Party/FreeRTOS/Source/tasks.o
                0x0000000008009720                pvTaskIncrementMutexHeldCount
 .text.prvAddCurrentTaskToDelayedList
                0x0000000008009748       0xa8 Middlewares/Third_Party/FreeRTOS/Source/tasks.o
 .text.xTimerCreateTimerTask
                0x00000000080097f0       0x90 Middlewares/Third_Party/FreeRTOS/Source/timers.o
                0x00000000080097f0                xTimerCreateTimerTask
 .text.xTimerCreate
                0x0000000008009880       0x42 Middlewares/Third_Party/FreeRTOS/Source/timers.o
                0x0000000008009880                xTimerCreate
 .text.xTimerCreateStatic
                0x00000000080098c2       0x78 Middlewares/Third_Party/FreeRTOS/Source/timers.o
                0x00000000080098c2                xTimerCreateStatic
 .text.prvInitialiseNewTimer
                0x000000000800993a       0x74 Middlewares/Third_Party/FreeRTOS/Source/timers.o
 *fill*         0x00000000080099ae        0x2 
 .text.xTimerGenericCommand
                0x00000000080099b0       0x98 Middlewares/Third_Party/FreeRTOS/Source/timers.o
                0x00000000080099b0                xTimerGenericCommand
 .text.prvProcessExpiredTimer
                0x0000000008009a48       0x98 Middlewares/Third_Party/FreeRTOS/Source/timers.o
 .text.prvTimerTask
                0x0000000008009ae0       0x24 Middlewares/Third_Party/FreeRTOS/Source/timers.o
 .text.prvProcessTimerOrBlockTask
                0x0000000008009b04       0x9c Middlewares/Third_Party/FreeRTOS/Source/timers.o
 .text.prvGetNextExpireTime
                0x0000000008009ba0       0x48 Middlewares/Third_Party/FreeRTOS/Source/timers.o
 .text.prvSampleTimeNow
                0x0000000008009be8       0x40 Middlewares/Third_Party/FreeRTOS/Source/timers.o
 .text.prvInsertTimerInActiveList
                0x0000000008009c28       0x84 Middlewares/Third_Party/FreeRTOS/Source/timers.o
 .text.prvProcessReceivedCommands
                0x0000000008009cac      0x1b8 Middlewares/Third_Party/FreeRTOS/Source/timers.o
 .text.prvSwitchTimerLists
                0x0000000008009e64       0xc8 Middlewares/Third_Party/FreeRTOS/Source/timers.o
 .text.prvCheckForValidListAndQueue
                0x0000000008009f2c       0x80 Middlewares/Third_Party/FreeRTOS/Source/timers.o
 .text.pvTimerGetTimerID
                0x0000000008009fac       0x3e Middlewares/Third_Party/FreeRTOS/Source/timers.o
                0x0000000008009fac                pvTimerGetTimerID
 *fill*         0x0000000008009fea        0x2 
 .text.pxPortInitialiseStack
                0x0000000008009fec       0x68 Middlewares/Third_Party/FreeRTOS/Source/portable/GCC/ARM_CM4F/port.o
                0x0000000008009fec                pxPortInitialiseStack
 .text.prvTaskExitError
                0x000000000800a054       0x54 Middlewares/Third_Party/FreeRTOS/Source/portable/GCC/ARM_CM4F/port.o
 *fill*         0x000000000800a0a8        0x8 
 .text.SVC_Handler
                0x000000000800a0b0       0x28 Middlewares/Third_Party/FreeRTOS/Source/portable/GCC/ARM_CM4F/port.o
                0x000000000800a0b0                SVC_Handler
 .text.prvPortStartFirstTask
                0x000000000800a0d8       0x28 Middlewares/Third_Party/FreeRTOS/Source/portable/GCC/ARM_CM4F/port.o
 .text.xPortStartScheduler
                0x000000000800a100      0x13c Middlewares/Third_Party/FreeRTOS/Source/portable/GCC/ARM_CM4F/port.o
                0x000000000800a100                xPortStartScheduler
 .text.vPortEnterCritical
                0x000000000800a23c       0x5c Middlewares/Third_Party/FreeRTOS/Source/portable/GCC/ARM_CM4F/port.o
                0x000000000800a23c                vPortEnterCritical
 .text.vPortExitCritical
                0x000000000800a298       0x50 Middlewares/Third_Party/FreeRTOS/Source/portable/GCC/ARM_CM4F/port.o
                0x000000000800a298                vPortExitCritical
 *fill*         0x000000000800a2e8        0x8 
 .text.PendSV_Handler
                0x000000000800a2f0       0x68 Middlewares/Third_Party/FreeRTOS/Source/portable/GCC/ARM_CM4F/port.o
                0x000000000800a2f0                PendSV_Handler
 .text.SysTick_Handler
                0x000000000800a358       0x40 Middlewares/Third_Party/FreeRTOS/Source/portable/GCC/ARM_CM4F/port.o
                0x000000000800a358                SysTick_Handler
 .text.vPortSetupTimerInterrupt
                0x000000000800a398       0x48 Middlewares/Third_Party/FreeRTOS/Source/portable/GCC/ARM_CM4F/port.o
                0x000000000800a398                vPortSetupTimerInterrupt
 .text.vPortEnableVFP
                0x000000000800a3e0       0x14 Middlewares/Third_Party/FreeRTOS/Source/portable/GCC/ARM_CM4F/port.o
 .text.vPortValidateInterruptPriority
                0x000000000800a3f4       0x7c Middlewares/Third_Party/FreeRTOS/Source/portable/GCC/ARM_CM4F/port.o
                0x000000000800a3f4                vPortValidateInterruptPriority
 .text.pvPortMalloc
                0x000000000800a470      0x184 Middlewares/Third_Party/FreeRTOS/Source/portable/MemMang/heap_4.o
                0x000000000800a470                pvPortMalloc
 .text.vPortFree
                0x000000000800a5f4       0xb0 Middlewares/Third_Party/FreeRTOS/Source/portable/MemMang/heap_4.o
                0x000000000800a5f4                vPortFree
 .text.prvHeapInit
                0x000000000800a6a4       0xc4 Middlewares/Third_Party/FreeRTOS/Source/portable/MemMang/heap_4.o
 .text.prvInsertBlockIntoFreeList
                0x000000000800a768       0xb4 Middlewares/Third_Party/FreeRTOS/Source/portable/MemMang/heap_4.o
 .text.__libc_init_array
                0x000000000800a81c       0x48 d:/stm32cubeide_1.5.0/stm32cubeide/plugins/com.st.stm32cube.ide.mcu.externaltools.gnu-tools-for-stm32.7-2018-q2-update.win32_1.5.0.202011040924/tools/bin/../lib/gcc/arm-none-eabi/7.3.1/../../../../arm-none-eabi/lib/thumb/v7e-m/fpv4-sp/hard\libc_nano.a(lib_a-init.o)
                0x000000000800a81c                __libc_init_array
 .text.memcpy   0x000000000800a864       0x16 d:/stm32cubeide_1.5.0/stm32cubeide/plugins/com.st.stm32cube.ide.mcu.externaltools.gnu-tools-for-stm32.7-2018-q2-update.win32_1.5.0.202011040924/tools/bin/../lib/gcc/arm-none-eabi/7.3.1/../../../../arm-none-eabi/lib/thumb/v7e-m/fpv4-sp/hard\libc_nano.a(lib_a-memcpy-stub.o)
                0x000000000800a864                memcpy
 .text.memset   0x000000000800a87a       0x10 d:/stm32cubeide_1.5.0/stm32cubeide/plugins/com.st.stm32cube.ide.mcu.externaltools.gnu-tools-for-stm32.7-2018-q2-update.win32_1.5.0.202011040924/tools/bin/../lib/gcc/arm-none-eabi/7.3.1/../../../../arm-none-eabi/lib/thumb/v7e-m/fpv4-sp/hard\libc_nano.a(lib_a-memset.o)
                0x000000000800a87a                memset
 *(.glue_7)
 .glue_7        0x000000000800a88a        0x0 linker stubs
 *(.glue_7t)
 .glue_7t       0x000000000800a88a        0x0 linker stubs
 *(.eh_frame)
 *fill*         0x000000000800a88a        0x2 
 .eh_frame      0x000000000800a88c        0x0 d:/stm32cubeide_1.5.0/stm32cubeide/plugins/com.st.stm32cube.ide.mcu.externaltools.gnu-tools-for-stm32.7-2018-q2-update.win32_1.5.0.202011040924/tools/bin/../lib/gcc/arm-none-eabi/7.3.1/thumb/v7e-m/fpv4-sp/hard/crtbegin.o
 *(.init)
 .init          0x000000000800a88c        0x4 d:/stm32cubeide_1.5.0/stm32cubeide/plugins/com.st.stm32cube.ide.mcu.externaltools.gnu-tools-for-stm32.7-2018-q2-update.win32_1.5.0.202011040924/tools/bin/../lib/gcc/arm-none-eabi/7.3.1/thumb/v7e-m/fpv4-sp/hard/crti.o
                0x000000000800a88c                _init
 .init          0x000000000800a890        0x8 d:/stm32cubeide_1.5.0/stm32cubeide/plugins/com.st.stm32cube.ide.mcu.externaltools.gnu-tools-for-stm32.7-2018-q2-update.win32_1.5.0.202011040924/tools/bin/../lib/gcc/arm-none-eabi/7.3.1/thumb/v7e-m/fpv4-sp/hard/crtn.o
 *(.fini)
 .fini          0x000000000800a898        0x4 d:/stm32cubeide_1.5.0/stm32cubeide/plugins/com.st.stm32cube.ide.mcu.externaltools.gnu-tools-for-stm32.7-2018-q2-update.win32_1.5.0.202011040924/tools/bin/../lib/gcc/arm-none-eabi/7.3.1/thumb/v7e-m/fpv4-sp/hard/crti.o
                0x000000000800a898                _fini
 .fini          0x000000000800a89c        0x8 d:/stm32cubeide_1.5.0/stm32cubeide/plugins/com.st.stm32cube.ide.mcu.externaltools.gnu-tools-for-stm32.7-2018-q2-update.win32_1.5.0.202011040924/tools/bin/../lib/gcc/arm-none-eabi/7.3.1/thumb/v7e-m/fpv4-sp/hard/crtn.o
                0x000000000800a8a4                . = ALIGN (0x4)
                0x000000000800a8a4                _etext = .

.vfp11_veneer   0x000000000800a8a4        0x0
 .vfp11_veneer  0x000000000800a8a4        0x0 linker stubs

.v4_bx          0x000000000800a8a4        0x0
 .v4_bx         0x000000000800a8a4        0x0 linker stubs

.iplt           0x000000000800a8a4        0x0
 .iplt          0x000000000800a8a4        0x0 d:/stm32cubeide_1.5.0/stm32cubeide/plugins/com.st.stm32cube.ide.mcu.externaltools.gnu-tools-for-stm32.7-2018-q2-update.win32_1.5.0.202011040924/tools/bin/../lib/gcc/arm-none-eabi/7.3.1/thumb/v7e-m/fpv4-sp/hard/crtbegin.o

.rodata         0x000000000800a8a8      0x418
                0x000000000800a8a8                . = ALIGN (0x4)
 *(.rodata)
 .rodata        0x000000000800a8a8       0xcb Core/Src/freertos.o
 *fill*         0x000000000800a973        0x1 
 .rodata        0x000000000800a974       0x18 Core/Src/printf.o
 .rodata        0x000000000800a98c        0x5 Middlewares/Third_Party/FreeRTOS/Source/tasks.o
 *fill*         0x000000000800a991        0x3 
 .rodata        0x000000000800a994        0xd Middlewares/Third_Party/FreeRTOS/Source/timers.o
 *(.rodata*)
 *fill*         0x000000000800a9a1        0x3 
 .rodata.font_8x5
                0x000000000800a9a4      0x1dd Core/Src/freertos.o
                0x000000000800a9a4                font_8x5
 *fill*         0x000000000800ab81        0x3 
 .rodata.HeartbeatTask_attributes
                0x000000000800ab84       0x24 Core/Src/freertos.o
                0x000000000800ab84                HeartbeatTask_attributes
 .rodata.Bmp280Task_attributes
                0x000000000800aba8       0x24 Core/Src/freertos.o
                0x000000000800aba8                Bmp280Task_attributes
 .rodata.OledTask_attributes
                0x000000000800abcc       0x24 Core/Src/freertos.o
                0x000000000800abcc                OledTask_attributes
 .rodata.QueueBmpData_attributes
                0x000000000800abf0       0x18 Core/Src/freertos.o
                0x000000000800abf0                QueueBmpData_attributes
 .rodata.TimerBmpData_attributes
                0x000000000800ac08       0x10 Core/Src/freertos.o
                0x000000000800ac08                TimerBmpData_attributes
 .rodata.MutexPrintf_attributes
                0x000000000800ac18       0x10 Core/Src/freertos.o
                0x000000000800ac18                MutexPrintf_attributes
 .rodata.MutexI2C1_attributes
                0x000000000800ac28       0x10 Core/Src/freertos.o
                0x000000000800ac28                MutexI2C1_attributes
 .rodata.MutexBmpData_attributes
                0x000000000800ac38       0x10 Core/Src/freertos.o
                0x000000000800ac38                MutexBmpData_attributes
 .rodata.SemaphoreBmpQueue_attributes
                0x000000000800ac48       0x10 Core/Src/freertos.o
                0x000000000800ac48                SemaphoreBmpQueue_attributes
 .rodata.pow10.5604
                0x000000000800ac58       0x50 Core/Src/printf.o
 .rodata.AHBPrescTable
                0x000000000800aca8       0x10 Core/Src/system_stm32f4xx.o
                0x000000000800aca8                AHBPrescTable
 .rodata.APBPrescTable
                0x000000000800acb8        0x8 Core/Src/system_stm32f4xx.o
                0x000000000800acb8                APBPrescTable
                0x000000000800acc0                . = ALIGN (0x4)

.ARM.extab      0x000000000800acc0        0x0
                0x000000000800acc0                . = ALIGN (0x4)
 *(.ARM.extab* .gnu.linkonce.armextab.*)
                0x000000000800acc0                . = ALIGN (0x4)

.ARM            0x000000000800acc0        0x8
                0x000000000800acc0                . = ALIGN (0x4)
                0x000000000800acc0                __exidx_start = .
 *(.ARM.exidx*)
 .ARM.exidx     0x000000000800acc0        0x8 d:/stm32cubeide_1.5.0/stm32cubeide/plugins/com.st.stm32cube.ide.mcu.externaltools.gnu-tools-for-stm32.7-2018-q2-update.win32_1.5.0.202011040924/tools/bin/../lib/gcc/arm-none-eabi/7.3.1/thumb/v7e-m/fpv4-sp/hard\libgcc.a(_udivmoddi4.o)
                0x000000000800acc8                __exidx_end = .
                0x000000000800acc8                . = ALIGN (0x4)

.rel.dyn        0x000000000800acc8        0x0
 .rel.iplt      0x000000000800acc8        0x0 d:/stm32cubeide_1.5.0/stm32cubeide/plugins/com.st.stm32cube.ide.mcu.externaltools.gnu-tools-for-stm32.7-2018-q2-update.win32_1.5.0.202011040924/tools/bin/../lib/gcc/arm-none-eabi/7.3.1/thumb/v7e-m/fpv4-sp/hard/crtbegin.o

.preinit_array  0x000000000800acc8        0x0
                0x000000000800acc8                . = ALIGN (0x4)
                0x000000000800acc8                PROVIDE (__preinit_array_start = .)
 *(.preinit_array*)
                0x000000000800acc8                PROVIDE (__preinit_array_end = .)
                0x000000000800acc8                . = ALIGN (0x4)

.init_array     0x000000000800acc8        0x4
                0x000000000800acc8                . = ALIGN (0x4)
                0x000000000800acc8                PROVIDE (__init_array_start = .)
 *(SORT_BY_NAME(.init_array.*))
 *(.init_array*)
 .init_array    0x000000000800acc8        0x4 d:/stm32cubeide_1.5.0/stm32cubeide/plugins/com.st.stm32cube.ide.mcu.externaltools.gnu-tools-for-stm32.7-2018-q2-update.win32_1.5.0.202011040924/tools/bin/../lib/gcc/arm-none-eabi/7.3.1/thumb/v7e-m/fpv4-sp/hard/crtbegin.o
                0x000000000800accc                PROVIDE (__init_array_end = .)
                0x000000000800accc                . = ALIGN (0x4)

.fini_array     0x000000000800accc        0x4
                0x000000000800accc                . = ALIGN (0x4)
                [!provide]                        PROVIDE (__fini_array_start = .)
 *(SORT_BY_NAME(.fini_array.*))
 *(.fini_array*)
 .fini_array    0x000000000800accc        0x4 d:/stm32cubeide_1.5.0/stm32cubeide/plugins/com.st.stm32cube.ide.mcu.externaltools.gnu-tools-for-stm32.7-2018-q2-update.win32_1.5.0.202011040924/tools/bin/../lib/gcc/arm-none-eabi/7.3.1/thumb/v7e-m/fpv4-sp/hard/crtbegin.o
                [!provide]                        PROVIDE (__fini_array_end = .)
                0x000000000800acd0                . = ALIGN (0x4)
                0x000000000800acd0                _sidata = LOADADDR (.data)

.data           0x0000000020000000       0x14 load address 0x000000000800acd0
                0x0000000020000000                . = ALIGN (0x4)
                0x0000000020000000                _sdata = .
 *(.data)
 *(.data*)
 .data.size     0x0000000020000000        0x1 Core/Src/GFX_BW.o
                0x0000000020000000                size
 *fill*         0x0000000020000001        0x3 
 .data.SystemCoreClock
                0x0000000020000004        0x4 Core/Src/system_stm32f4xx.o
                0x0000000020000004                SystemCoreClock
 .data.uwTickPrio
                0x0000000020000008        0x4 Drivers/STM32F4xx_HAL_Driver/Src/stm32f4xx_hal.o
                0x0000000020000008                uwTickPrio
 .data.uwTickFreq
                0x000000002000000c        0x1 Drivers/STM32F4xx_HAL_Driver/Src/stm32f4xx_hal.o
                0x000000002000000c                uwTickFreq
 *fill*         0x000000002000000d        0x3 
 .data.uxCriticalNesting
                0x0000000020000010        0x4 Middlewares/Third_Party/FreeRTOS/Source/portable/GCC/ARM_CM4F/port.o
 *(.RamFunc)
 *(.RamFunc*)
                0x0000000020000014                . = ALIGN (0x4)
                0x0000000020000014                _edata = .

.igot.plt       0x0000000020000014        0x0 load address 0x000000000800ace4
 .igot.plt      0x0000000020000014        0x0 d:/stm32cubeide_1.5.0/stm32cubeide/plugins/com.st.stm32cube.ide.mcu.externaltools.gnu-tools-for-stm32.7-2018-q2-update.win32_1.5.0.202011040924/tools/bin/../lib/gcc/arm-none-eabi/7.3.1/thumb/v7e-m/fpv4-sp/hard/crtbegin.o
                0x0000000020000014                . = ALIGN (0x4)

.bss            0x0000000020000014     0x4e68 load address 0x000000000800ace4
                0x0000000020000014                _sbss = .
                0x0000000020000014                __bss_start__ = _sbss
 *(.bss)
 .bss           0x0000000020000014       0x1c d:/stm32cubeide_1.5.0/stm32cubeide/plugins/com.st.stm32cube.ide.mcu.externaltools.gnu-tools-for-stm32.7-2018-q2-update.win32_1.5.0.202011040924/tools/bin/../lib/gcc/arm-none-eabi/7.3.1/thumb/v7e-m/fpv4-sp/hard/crtbegin.o
 *(.bss*)
 .bss.buffer    0x0000000020000030      0x400 Core/Src/SSD1306_OLED.o
 .bss.KernelState
                0x0000000020000430        0x4 Middlewares/Third_Party/FreeRTOS/Source/CMSIS_RTOS_V2/cmsis_os2.o
 .bss.Idle_TCB  0x0000000020000434       0x5c Middlewares/Third_Party/FreeRTOS/Source/CMSIS_RTOS_V2/cmsis_os2.o
 .bss.Idle_Stack
                0x0000000020000490      0x200 Middlewares/Third_Party/FreeRTOS/Source/CMSIS_RTOS_V2/cmsis_os2.o
 .bss.Timer_TCB
                0x0000000020000690       0x5c Middlewares/Third_Party/FreeRTOS/Source/CMSIS_RTOS_V2/cmsis_os2.o
 .bss.Timer_Stack
                0x00000000200006ec      0x400 Middlewares/Third_Party/FreeRTOS/Source/CMSIS_RTOS_V2/cmsis_os2.o
 .bss.pxCurrentTCB
                0x0000000020000aec        0x4 Middlewares/Third_Party/FreeRTOS/Source/tasks.o
                0x0000000020000aec                pxCurrentTCB
 .bss.pxReadyTasksLists
                0x0000000020000af0      0x460 Middlewares/Third_Party/FreeRTOS/Source/tasks.o
 .bss.xDelayedTaskList1
                0x0000000020000f50       0x14 Middlewares/Third_Party/FreeRTOS/Source/tasks.o
 .bss.xDelayedTaskList2
                0x0000000020000f64       0x14 Middlewares/Third_Party/FreeRTOS/Source/tasks.o
 .bss.pxDelayedTaskList
                0x0000000020000f78        0x4 Middlewares/Third_Party/FreeRTOS/Source/tasks.o
 .bss.pxOverflowDelayedTaskList
                0x0000000020000f7c        0x4 Middlewares/Third_Party/FreeRTOS/Source/tasks.o
 .bss.xPendingReadyList
                0x0000000020000f80       0x14 Middlewares/Third_Party/FreeRTOS/Source/tasks.o
 .bss.xTasksWaitingTermination
                0x0000000020000f94       0x14 Middlewares/Third_Party/FreeRTOS/Source/tasks.o
 .bss.uxDeletedTasksWaitingCleanUp
                0x0000000020000fa8        0x4 Middlewares/Third_Party/FreeRTOS/Source/tasks.o
 .bss.xSuspendedTaskList
                0x0000000020000fac       0x14 Middlewares/Third_Party/FreeRTOS/Source/tasks.o
 .bss.uxCurrentNumberOfTasks
                0x0000000020000fc0        0x4 Middlewares/Third_Party/FreeRTOS/Source/tasks.o
 .bss.xTickCount
                0x0000000020000fc4        0x4 Middlewares/Third_Party/FreeRTOS/Source/tasks.o
 .bss.uxTopReadyPriority
                0x0000000020000fc8        0x4 Middlewares/Third_Party/FreeRTOS/Source/tasks.o
 .bss.xSchedulerRunning
                0x0000000020000fcc        0x4 Middlewares/Third_Party/FreeRTOS/Source/tasks.o
 .bss.uxPendedTicks
                0x0000000020000fd0        0x4 Middlewares/Third_Party/FreeRTOS/Source/tasks.o
 .bss.xYieldPending
                0x0000000020000fd4        0x4 Middlewares/Third_Party/FreeRTOS/Source/tasks.o
 .bss.xNumOfOverflows
                0x0000000020000fd8        0x4 Middlewares/Third_Party/FreeRTOS/Source/tasks.o
 .bss.uxTaskNumber
                0x0000000020000fdc        0x4 Middlewares/Third_Party/FreeRTOS/Source/tasks.o
 .bss.xNextTaskUnblockTime
                0x0000000020000fe0        0x4 Middlewares/Third_Party/FreeRTOS/Source/tasks.o
 .bss.xIdleTaskHandle
                0x0000000020000fe4        0x4 Middlewares/Third_Party/FreeRTOS/Source/tasks.o
 .bss.uxSchedulerSuspended
                0x0000000020000fe8        0x4 Middlewares/Third_Party/FreeRTOS/Source/tasks.o
 .bss.xActiveTimerList1
                0x0000000020000fec       0x14 Middlewares/Third_Party/FreeRTOS/Source/timers.o
 .bss.xActiveTimerList2
                0x0000000020001000       0x14 Middlewares/Third_Party/FreeRTOS/Source/timers.o
 .bss.pxCurrentTimerList
                0x0000000020001014        0x4 Middlewares/Third_Party/FreeRTOS/Source/timers.o
 .bss.pxOverflowTimerList
                0x0000000020001018        0x4 Middlewares/Third_Party/FreeRTOS/Source/timers.o
 .bss.xTimerQueue
                0x000000002000101c        0x4 Middlewares/Third_Party/FreeRTOS/Source/timers.o
 .bss.xTimerTaskHandle
                0x0000000020001020        0x4 Middlewares/Third_Party/FreeRTOS/Source/timers.o
 .bss.xLastTime.6741
                0x0000000020001024        0x4 Middlewares/Third_Party/FreeRTOS/Source/timers.o
 .bss.ucStaticTimerQueueStorage.6792
                0x0000000020001028       0xa0 Middlewares/Third_Party/FreeRTOS/Source/timers.o
 .bss.xStaticTimerQueue.6791
                0x00000000200010c8       0x50 Middlewares/Third_Party/FreeRTOS/Source/timers.o
 .bss.ucMaxSysCallPriority
                0x0000000020001118        0x1 Middlewares/Third_Party/FreeRTOS/Source/portable/GCC/ARM_CM4F/port.o
 *fill*         0x0000000020001119        0x3 
 .bss.ulMaxPRIGROUPValue
                0x000000002000111c        0x4 Middlewares/Third_Party/FreeRTOS/Source/portable/GCC/ARM_CM4F/port.o
 .bss.ucHeap    0x0000000020001120     0x3c00 Middlewares/Third_Party/FreeRTOS/Source/portable/MemMang/heap_4.o
 .bss.xStart    0x0000000020004d20        0x8 Middlewares/Third_Party/FreeRTOS/Source/portable/MemMang/heap_4.o
 .bss.pxEnd     0x0000000020004d28        0x4 Middlewares/Third_Party/FreeRTOS/Source/portable/MemMang/heap_4.o
 .bss.xFreeBytesRemaining
                0x0000000020004d2c        0x4 Middlewares/Third_Party/FreeRTOS/Source/portable/MemMang/heap_4.o
 .bss.xMinimumEverFreeBytesRemaining
                0x0000000020004d30        0x4 Middlewares/Third_Party/FreeRTOS/Source/portable/MemMang/heap_4.o
 .bss.xBlockAllocatedBit
                0x0000000020004d34        0x4 Middlewares/Third_Party/FreeRTOS/Source/portable/MemMang/heap_4.o
 *(COMMON)
 COMMON         0x0000000020004d38        0x4 Core/Src/GFX_BW.o
                0x0000000020004d38                font
 COMMON         0x0000000020004d3c        0x4 Core/Src/SSD1306_OLED.o
                0x0000000020004d3c                oled_i2c
 COMMON         0x0000000020004d40       0x24 Core/Src/freertos.o
                0x0000000020004d40                TimerBmpDataHandle
                0x0000000020004d44                SemaphoreBmpQueueHandle
                0x0000000020004d48                OledTaskHandle
                0x0000000020004d4c                QueueBmpDataHandle
                0x0000000020004d50                MutexPrintfHandle
                0x0000000020004d54                MutexI2C1Handle
                0x0000000020004d58                Bmp280TaskHandle
                0x0000000020004d5c                MutexBmpDataHandle
                0x0000000020004d60                HeartbeatTaskHandle
 COMMON         0x0000000020004d64       0x54 Core/Src/i2c.o
                0x0000000020004d64                hi2c1
 COMMON         0x0000000020004db8       0x40 Core/Src/stm32f4xx_hal_timebase_tim.o
                0x0000000020004db8                htim10
 COMMON         0x0000000020004df8       0x40 Core/Src/usart.o
                0x0000000020004df8                huart2
 COMMON         0x0000000020004e38        0x4 Drivers/STM32F4xx_HAL_Driver/Src/stm32f4xx_hal.o
                0x0000000020004e38                uwTick
 COMMON         0x0000000020004e3c       0x40 Middlewares/Third_Party/FreeRTOS/Source/queue.o
                0x0000000020004e3c                xQueueRegistry
                0x0000000020004e7c                . = ALIGN (0x4)
                0x0000000020004e7c                _ebss = .
                0x0000000020004e7c                __bss_end__ = _ebss

._user_heap_stack
                0x0000000020004e7c      0x604 load address 0x000000000800ace4
                0x0000000020004e80                . = ALIGN (0x8)
 *fill*         0x0000000020004e7c        0x4 
                [!provide]                        PROVIDE (end = .)
                0x0000000020004e80                PROVIDE (_end = .)
                0x0000000020005080                . = (. + _Min_Heap_Size)
 *fill*         0x0000000020004e80      0x200 
                0x0000000020005480                . = (. + _Min_Stack_Size)
 *fill*         0x0000000020005080      0x400 
                0x0000000020005480                . = ALIGN (0x8)

/DISCARD/
 libc.a(*)
 libm.a(*)
 libgcc.a(*)

.ARM.attributes
                0x0000000000000000       0x30
 *(.ARM.attributes)
 .ARM.attributes
                0x0000000000000000       0x22 d:/stm32cubeide_1.5.0/stm32cubeide/plugins/com.st.stm32cube.ide.mcu.externaltools.gnu-tools-for-stm32.7-2018-q2-update.win32_1.5.0.202011040924/tools/bin/../lib/gcc/arm-none-eabi/7.3.1/thumb/v7e-m/fpv4-sp/hard/crti.o
 .ARM.attributes
                0x0000000000000022       0x34 d:/stm32cubeide_1.5.0/stm32cubeide/plugins/com.st.stm32cube.ide.mcu.externaltools.gnu-tools-for-stm32.7-2018-q2-update.win32_1.5.0.202011040924/tools/bin/../lib/gcc/arm-none-eabi/7.3.1/thumb/v7e-m/fpv4-sp/hard/crtbegin.o
 .ARM.attributes
                0x0000000000000056       0x39 Core/Src/GFX_BW.o
 .ARM.attributes
                0x000000000000008f       0x39 Core/Src/SSD1306_OLED.o
 .ARM.attributes
                0x00000000000000c8       0x39 Core/Src/bmp280.o
 .ARM.attributes
                0x0000000000000101       0x39 Core/Src/freertos.o
 .ARM.attributes
                0x000000000000013a       0x39 Core/Src/gpio.o
 .ARM.attributes
                0x0000000000000173       0x39 Core/Src/i2c.o
 .ARM.attributes
                0x00000000000001ac       0x39 Core/Src/main.o
 .ARM.attributes
                0x00000000000001e5       0x39 Core/Src/printf.o
 .ARM.attributes
                0x000000000000021e       0x39 Core/Src/stm32f4xx_hal_msp.o
 .ARM.attributes
                0x0000000000000257       0x39 Core/Src/stm32f4xx_hal_timebase_tim.o
 .ARM.attributes
                0x0000000000000290       0x39 Core/Src/stm32f4xx_it.o
 .ARM.attributes
                0x00000000000002c9       0x39 Core/Src/system_stm32f4xx.o
 .ARM.attributes
                0x0000000000000302       0x39 Core/Src/usart.o
 .ARM.attributes
                0x000000000000033b       0x21 Core/Startup/startup_stm32f411retx.o
 .ARM.attributes
                0x000000000000035c       0x39 Drivers/STM32F4xx_HAL_Driver/Src/stm32f4xx_hal.o
 .ARM.attributes
                0x0000000000000395       0x39 Drivers/STM32F4xx_HAL_Driver/Src/stm32f4xx_hal_cortex.o
 .ARM.attributes
                0x00000000000003ce       0x39 Drivers/STM32F4xx_HAL_Driver/Src/stm32f4xx_hal_gpio.o
 .ARM.attributes
                0x0000000000000407       0x39 Drivers/STM32F4xx_HAL_Driver/Src/stm32f4xx_hal_i2c.o
 .ARM.attributes
                0x0000000000000440       0x39 Drivers/STM32F4xx_HAL_Driver/Src/stm32f4xx_hal_rcc.o
 .ARM.attributes
                0x0000000000000479       0x39 Drivers/STM32F4xx_HAL_Driver/Src/stm32f4xx_hal_tim.o
 .ARM.attributes
                0x00000000000004b2       0x39 Drivers/STM32F4xx_HAL_Driver/Src/stm32f4xx_hal_tim_ex.o
 .ARM.attributes
                0x00000000000004eb       0x39 Drivers/STM32F4xx_HAL_Driver/Src/stm32f4xx_hal_uart.o
 .ARM.attributes
                0x0000000000000524       0x39 Middlewares/Third_Party/FreeRTOS/Source/CMSIS_RTOS_V2/cmsis_os2.o
 .ARM.attributes
                0x000000000000055d       0x39 Middlewares/Third_Party/FreeRTOS/Source/list.o
 .ARM.attributes
                0x0000000000000596       0x39 Middlewares/Third_Party/FreeRTOS/Source/queue.o
 .ARM.attributes
                0x00000000000005cf       0x39 Middlewares/Third_Party/FreeRTOS/Source/tasks.o
 .ARM.attributes
                0x0000000000000608       0x39 Middlewares/Third_Party/FreeRTOS/Source/timers.o
 .ARM.attributes
                0x0000000000000641       0x39 Middlewares/Third_Party/FreeRTOS/Source/portable/GCC/ARM_CM4F/port.o
 .ARM.attributes
                0x000000000000067a       0x39 Middlewares/Third_Party/FreeRTOS/Source/portable/MemMang/heap_4.o
 .ARM.attributes
                0x00000000000006b3       0x34 d:/stm32cubeide_1.5.0/stm32cubeide/plugins/com.st.stm32cube.ide.mcu.externaltools.gnu-tools-for-stm32.7-2018-q2-update.win32_1.5.0.202011040924/tools/bin/../lib/gcc/arm-none-eabi/7.3.1/../../../../arm-none-eabi/lib/thumb/v7e-m/fpv4-sp/hard\libc_nano.a(lib_a-init.o)
 .ARM.attributes
                0x00000000000006e7       0x34 d:/stm32cubeide_1.5.0/stm32cubeide/plugins/com.st.stm32cube.ide.mcu.externaltools.gnu-tools-for-stm32.7-2018-q2-update.win32_1.5.0.202011040924/tools/bin/../lib/gcc/arm-none-eabi/7.3.1/../../../../arm-none-eabi/lib/thumb/v7e-m/fpv4-sp/hard\libc_nano.a(lib_a-memcpy-stub.o)
 .ARM.attributes
                0x000000000000071b       0x34 d:/stm32cubeide_1.5.0/stm32cubeide/plugins/com.st.stm32cube.ide.mcu.externaltools.gnu-tools-for-stm32.7-2018-q2-update.win32_1.5.0.202011040924/tools/bin/../lib/gcc/arm-none-eabi/7.3.1/../../../../arm-none-eabi/lib/thumb/v7e-m/fpv4-sp/hard\libc_nano.a(lib_a-memset.o)
 .ARM.attributes
                0x000000000000074f       0x22 d:/stm32cubeide_1.5.0/stm32cubeide/plugins/com.st.stm32cube.ide.mcu.externaltools.gnu-tools-for-stm32.7-2018-q2-update.win32_1.5.0.202011040924/tools/bin/../lib/gcc/arm-none-eabi/7.3.1/thumb/v7e-m/fpv4-sp/hard\libgcc.a(_arm_addsubdf3.o)
 .ARM.attributes
                0x0000000000000771       0x22 d:/stm32cubeide_1.5.0/stm32cubeide/plugins/com.st.stm32cube.ide.mcu.externaltools.gnu-tools-for-stm32.7-2018-q2-update.win32_1.5.0.202011040924/tools/bin/../lib/gcc/arm-none-eabi/7.3.1/thumb/v7e-m/fpv4-sp/hard\libgcc.a(_arm_muldivdf3.o)
 .ARM.attributes
                0x0000000000000793       0x22 d:/stm32cubeide_1.5.0/stm32cubeide/plugins/com.st.stm32cube.ide.mcu.externaltools.gnu-tools-for-stm32.7-2018-q2-update.win32_1.5.0.202011040924/tools/bin/../lib/gcc/arm-none-eabi/7.3.1/thumb/v7e-m/fpv4-sp/hard\libgcc.a(_arm_cmpdf2.o)
 .ARM.attributes
                0x00000000000007b5       0x22 d:/stm32cubeide_1.5.0/stm32cubeide/plugins/com.st.stm32cube.ide.mcu.externaltools.gnu-tools-for-stm32.7-2018-q2-update.win32_1.5.0.202011040924/tools/bin/../lib/gcc/arm-none-eabi/7.3.1/thumb/v7e-m/fpv4-sp/hard\libgcc.a(_arm_fixdfsi.o)
 .ARM.attributes
                0x00000000000007d7       0x22 d:/stm32cubeide_1.5.0/stm32cubeide/plugins/com.st.stm32cube.ide.mcu.externaltools.gnu-tools-for-stm32.7-2018-q2-update.win32_1.5.0.202011040924/tools/bin/../lib/gcc/arm-none-eabi/7.3.1/thumb/v7e-m/fpv4-sp/hard\libgcc.a(_arm_fixunsdfsi.o)
 .ARM.attributes
                0x00000000000007f9       0x22 d:/stm32cubeide_1.5.0/stm32cubeide/plugins/com.st.stm32cube.ide.mcu.externaltools.gnu-tools-for-stm32.7-2018-q2-update.win32_1.5.0.202011040924/tools/bin/../lib/gcc/arm-none-eabi/7.3.1/thumb/v7e-m/fpv4-sp/hard\libgcc.a(_arm_truncdfsf2.o)
 .ARM.attributes
                0x000000000000081b       0x22 d:/stm32cubeide_1.5.0/stm32cubeide/plugins/com.st.stm32cube.ide.mcu.externaltools.gnu-tools-for-stm32.7-2018-q2-update.win32_1.5.0.202011040924/tools/bin/../lib/gcc/arm-none-eabi/7.3.1/thumb/v7e-m/fpv4-sp/hard\libgcc.a(_aeabi_uldivmod.o)
 .ARM.attributes
                0x000000000000083d       0x34 d:/stm32cubeide_1.5.0/stm32cubeide/plugins/com.st.stm32cube.ide.mcu.externaltools.gnu-tools-for-stm32.7-2018-q2-update.win32_1.5.0.202011040924/tools/bin/../lib/gcc/arm-none-eabi/7.3.1/thumb/v7e-m/fpv4-sp/hard\libgcc.a(_udivmoddi4.o)
 .ARM.attributes
                0x0000000000000871       0x22 d:/stm32cubeide_1.5.0/stm32cubeide/plugins/com.st.stm32cube.ide.mcu.externaltools.gnu-tools-for-stm32.7-2018-q2-update.win32_1.5.0.202011040924/tools/bin/../lib/gcc/arm-none-eabi/7.3.1/thumb/v7e-m/fpv4-sp/hard\libgcc.a(_dvmd_tls.o)
 .ARM.attributes
                0x0000000000000893       0x22 d:/stm32cubeide_1.5.0/stm32cubeide/plugins/com.st.stm32cube.ide.mcu.externaltools.gnu-tools-for-stm32.7-2018-q2-update.win32_1.5.0.202011040924/tools/bin/../lib/gcc/arm-none-eabi/7.3.1/thumb/v7e-m/fpv4-sp/hard/crtn.o
OUTPUT(T11_L53_RTOS_SimpleProject_Queue.elf elf32-littlearm)

.debug_info     0x0000000000000000    0x1e80e
 .debug_info    0x0000000000000000     0x1483 Core/Src/GFX_BW.o
 .debug_info    0x0000000000001483      0xfaa Core/Src/SSD1306_OLED.o
 .debug_info    0x000000000000242d      0xacd Core/Src/bmp280.o
 .debug_info    0x0000000000002efa     0x105f Core/Src/freertos.o
 .debug_info    0x0000000000003f59      0x4f2 Core/Src/gpio.o
 .debug_info    0x000000000000444b      0xa08 Core/Src/i2c.o
 .debug_info    0x0000000000004e53      0xef1 Core/Src/main.o
 .debug_info    0x0000000000005d44      0xd40 Core/Src/printf.o
 .debug_info    0x0000000000006a84      0x520 Core/Src/stm32f4xx_hal_msp.o
 .debug_info    0x0000000000006fa4      0xabf Core/Src/stm32f4xx_hal_timebase_tim.o
 .debug_info    0x0000000000007a63      0x6b0 Core/Src/stm32f4xx_it.o
 .debug_info    0x0000000000008113      0x57e Core/Src/system_stm32f4xx.o
 .debug_info    0x0000000000008691      0x96c Core/Src/usart.o
 .debug_info    0x0000000000008ffd       0x22 Core/Startup/startup_stm32f411retx.o
 .debug_info    0x000000000000901f      0x8d5 Drivers/STM32F4xx_HAL_Driver/Src/stm32f4xx_hal.o
 .debug_info    0x00000000000098f4      0xd98 Drivers/STM32F4xx_HAL_Driver/Src/stm32f4xx_hal_cortex.o
 .debug_info    0x000000000000a68c      0x7d7 Drivers/STM32F4xx_HAL_Driver/Src/stm32f4xx_hal_gpio.o
 .debug_info    0x000000000000ae63     0x242b Drivers/STM32F4xx_HAL_Driver/Src/stm32f4xx_hal_i2c.o
 .debug_info    0x000000000000d28e      0x92a Drivers/STM32F4xx_HAL_Driver/Src/stm32f4xx_hal_rcc.o
 .debug_info    0x000000000000dbb8     0x24a1 Drivers/STM32F4xx_HAL_Driver/Src/stm32f4xx_hal_tim.o
 .debug_info    0x0000000000010059     0x114f Drivers/STM32F4xx_HAL_Driver/Src/stm32f4xx_hal_tim_ex.o
 .debug_info    0x00000000000111a8     0x1244 Drivers/STM32F4xx_HAL_Driver/Src/stm32f4xx_hal_uart.o
 .debug_info    0x00000000000123ec     0x401f Middlewares/Third_Party/FreeRTOS/Source/CMSIS_RTOS_V2/cmsis_os2.o
 .debug_info    0x000000000001640b      0xacb Middlewares/Third_Party/FreeRTOS/Source/list.o
 .debug_info    0x0000000000016ed6     0x239c Middlewares/Third_Party/FreeRTOS/Source/queue.o
 .debug_info    0x0000000000019272     0x29c5 Middlewares/Third_Party/FreeRTOS/Source/tasks.o
 .debug_info    0x000000000001bc37     0x1aba Middlewares/Third_Party/FreeRTOS/Source/timers.o
 .debug_info    0x000000000001d6f1      0x533 Middlewares/Third_Party/FreeRTOS/Source/portable/GCC/ARM_CM4F/port.o
 .debug_info    0x000000000001dc24      0xbea Middlewares/Third_Party/FreeRTOS/Source/portable/MemMang/heap_4.o

.debug_abbrev   0x0000000000000000     0x3be4
 .debug_abbrev  0x0000000000000000      0x29a Core/Src/GFX_BW.o
 .debug_abbrev  0x000000000000029a      0x235 Core/Src/SSD1306_OLED.o
 .debug_abbrev  0x00000000000004cf      0x1b4 Core/Src/bmp280.o
 .debug_abbrev  0x0000000000000683      0x203 Core/Src/freertos.o
 .debug_abbrev  0x0000000000000886      0x134 Core/Src/gpio.o
 .debug_abbrev  0x00000000000009ba      0x199 Core/Src/i2c.o
 .debug_abbrev  0x0000000000000b53      0x1d7 Core/Src/main.o
 .debug_abbrev  0x0000000000000d2a      0x206 Core/Src/printf.o
 .debug_abbrev  0x0000000000000f30      0x112 Core/Src/stm32f4xx_hal_msp.o
 .debug_abbrev  0x0000000000001042      0x1ac Core/Src/stm32f4xx_hal_timebase_tim.o
 .debug_abbrev  0x00000000000011ee      0x169 Core/Src/stm32f4xx_it.o
 .debug_abbrev  0x0000000000001357      0x12b Core/Src/system_stm32f4xx.o
 .debug_abbrev  0x0000000000001482      0x199 Core/Src/usart.o
 .debug_abbrev  0x000000000000161b       0x12 Core/Startup/startup_stm32f411retx.o
 .debug_abbrev  0x000000000000162d      0x1f2 Drivers/STM32F4xx_HAL_Driver/Src/stm32f4xx_hal.o
 .debug_abbrev  0x000000000000181f      0x2fa Drivers/STM32F4xx_HAL_Driver/Src/stm32f4xx_hal_cortex.o
 .debug_abbrev  0x0000000000001b19      0x1c9 Drivers/STM32F4xx_HAL_Driver/Src/stm32f4xx_hal_gpio.o
 .debug_abbrev  0x0000000000001ce2      0x263 Drivers/STM32F4xx_HAL_Driver/Src/stm32f4xx_hal_i2c.o
 .debug_abbrev  0x0000000000001f45      0x245 Drivers/STM32F4xx_HAL_Driver/Src/stm32f4xx_hal_rcc.o
 .debug_abbrev  0x000000000000218a      0x23f Drivers/STM32F4xx_HAL_Driver/Src/stm32f4xx_hal_tim.o
 .debug_abbrev  0x00000000000023c9      0x22d Drivers/STM32F4xx_HAL_Driver/Src/stm32f4xx_hal_tim_ex.o
 .debug_abbrev  0x00000000000025f6      0x251 Drivers/STM32F4xx_HAL_Driver/Src/stm32f4xx_hal_uart.o
 .debug_abbrev  0x0000000000002847      0x3c3 Middlewares/Third_Party/FreeRTOS/Source/CMSIS_RTOS_V2/cmsis_os2.o
 .debug_abbrev  0x0000000000002c0a      0x1cf Middlewares/Third_Party/FreeRTOS/Source/list.o
 .debug_abbrev  0x0000000000002dd9      0x336 Middlewares/Third_Party/FreeRTOS/Source/queue.o
 .debug_abbrev  0x000000000000310f      0x350 Middlewares/Third_Party/FreeRTOS/Source/tasks.o
 .debug_abbrev  0x000000000000345f      0x2d7 Middlewares/Third_Party/FreeRTOS/Source/timers.o
 .debug_abbrev  0x0000000000003736      0x210 Middlewares/Third_Party/FreeRTOS/Source/portable/GCC/ARM_CM4F/port.o
 .debug_abbrev  0x0000000000003946      0x29e Middlewares/Third_Party/FreeRTOS/Source/portable/MemMang/heap_4.o

.debug_aranges  0x0000000000000000     0x17f0
 .debug_aranges
                0x0000000000000000       0xc8 Core/Src/GFX_BW.o
 .debug_aranges
                0x00000000000000c8       0x48 Core/Src/SSD1306_OLED.o
 .debug_aranges
                0x0000000000000110       0x78 Core/Src/bmp280.o
 .debug_aranges
                0x0000000000000188       0x48 Core/Src/freertos.o
 .debug_aranges
                0x00000000000001d0       0x20 Core/Src/gpio.o
 .debug_aranges
                0x00000000000001f0       0x30 Core/Src/i2c.o
 .debug_aranges
                0x0000000000000220       0x38 Core/Src/main.o
 .debug_aranges
                0x0000000000000258       0xb8 Core/Src/printf.o
 .debug_aranges
                0x0000000000000310       0x20 Core/Src/stm32f4xx_hal_msp.o
 .debug_aranges
                0x0000000000000330       0x30 Core/Src/stm32f4xx_hal_timebase_tim.o
 .debug_aranges
                0x0000000000000360       0x50 Core/Src/stm32f4xx_it.o
 .debug_aranges
                0x00000000000003b0       0x28 Core/Src/system_stm32f4xx.o
 .debug_aranges
                0x00000000000003d8       0x30 Core/Src/usart.o
 .debug_aranges
                0x0000000000000408       0x28 Core/Startup/startup_stm32f411retx.o
 .debug_aranges
                0x0000000000000430       0xf0 Drivers/STM32F4xx_HAL_Driver/Src/stm32f4xx_hal.o
 .debug_aranges
                0x0000000000000520      0x118 Drivers/STM32F4xx_HAL_Driver/Src/stm32f4xx_hal_cortex.o
 .debug_aranges
                0x0000000000000638       0x58 Drivers/STM32F4xx_HAL_Driver/Src/stm32f4xx_hal_gpio.o
 .debug_aranges
                0x0000000000000690      0x2a0 Drivers/STM32F4xx_HAL_Driver/Src/stm32f4xx_hal_i2c.o
 .debug_aranges
                0x0000000000000930       0x88 Drivers/STM32F4xx_HAL_Driver/Src/stm32f4xx_hal_rcc.o
 .debug_aranges
                0x00000000000009b8      0x3a8 Drivers/STM32F4xx_HAL_Driver/Src/stm32f4xx_hal_tim.o
 .debug_aranges
                0x0000000000000d60      0x150 Drivers/STM32F4xx_HAL_Driver/Src/stm32f4xx_hal_tim_ex.o
 .debug_aranges
                0x0000000000000eb0      0x1d0 Drivers/STM32F4xx_HAL_Driver/Src/stm32f4xx_hal_uart.o
 .debug_aranges
                0x0000000000001080      0x228 Middlewares/Third_Party/FreeRTOS/Source/CMSIS_RTOS_V2/cmsis_os2.o
 .debug_aranges
                0x00000000000012a8       0x40 Middlewares/Third_Party/FreeRTOS/Source/list.o
 .debug_aranges
                0x00000000000012e8      0x158 Middlewares/Third_Party/FreeRTOS/Source/queue.o
 .debug_aranges
                0x0000000000001440      0x1f8 Middlewares/Third_Party/FreeRTOS/Source/tasks.o
 .debug_aranges
                0x0000000000001638       0xe8 Middlewares/Third_Party/FreeRTOS/Source/timers.o
 .debug_aranges
                0x0000000000001720       0x80 Middlewares/Third_Party/FreeRTOS/Source/portable/GCC/ARM_CM4F/port.o
 .debug_aranges
                0x00000000000017a0       0x50 Middlewares/Third_Party/FreeRTOS/Source/portable/MemMang/heap_4.o

.debug_ranges   0x0000000000000000     0x1650
 .debug_ranges  0x0000000000000000       0xb8 Core/Src/GFX_BW.o
 .debug_ranges  0x00000000000000b8       0x38 Core/Src/SSD1306_OLED.o
 .debug_ranges  0x00000000000000f0       0x68 Core/Src/bmp280.o
 .debug_ranges  0x0000000000000158       0x38 Core/Src/freertos.o
 .debug_ranges  0x0000000000000190       0x10 Core/Src/gpio.o
 .debug_ranges  0x00000000000001a0       0x20 Core/Src/i2c.o
 .debug_ranges  0x00000000000001c0       0x28 Core/Src/main.o
 .debug_ranges  0x00000000000001e8       0xa8 Core/Src/printf.o
 .debug_ranges  0x0000000000000290       0x10 Core/Src/stm32f4xx_hal_msp.o
 .debug_ranges  0x00000000000002a0       0x20 Core/Src/stm32f4xx_hal_timebase_tim.o
 .debug_ranges  0x00000000000002c0       0x40 Core/Src/stm32f4xx_it.o
 .debug_ranges  0x0000000000000300       0x18 Core/Src/system_stm32f4xx.o
 .debug_ranges  0x0000000000000318       0x20 Core/Src/usart.o
 .debug_ranges  0x0000000000000338       0x20 Core/Startup/startup_stm32f411retx.o
 .debug_ranges  0x0000000000000358       0xe0 Drivers/STM32F4xx_HAL_Driver/Src/stm32f4xx_hal.o
 .debug_ranges  0x0000000000000438      0x108 Drivers/STM32F4xx_HAL_Driver/Src/stm32f4xx_hal_cortex.o
 .debug_ranges  0x0000000000000540       0x48 Drivers/STM32F4xx_HAL_Driver/Src/stm32f4xx_hal_gpio.o
 .debug_ranges  0x0000000000000588      0x2b8 Drivers/STM32F4xx_HAL_Driver/Src/stm32f4xx_hal_i2c.o
 .debug_ranges  0x0000000000000840       0x78 Drivers/STM32F4xx_HAL_Driver/Src/stm32f4xx_hal_rcc.o
 .debug_ranges  0x00000000000008b8      0x398 Drivers/STM32F4xx_HAL_Driver/Src/stm32f4xx_hal_tim.o
 .debug_ranges  0x0000000000000c50      0x140 Drivers/STM32F4xx_HAL_Driver/Src/stm32f4xx_hal_tim_ex.o
 .debug_ranges  0x0000000000000d90      0x1c0 Drivers/STM32F4xx_HAL_Driver/Src/stm32f4xx_hal_uart.o
 .debug_ranges  0x0000000000000f50      0x218 Middlewares/Third_Party/FreeRTOS/Source/CMSIS_RTOS_V2/cmsis_os2.o
 .debug_ranges  0x0000000000001168       0x30 Middlewares/Third_Party/FreeRTOS/Source/list.o
 .debug_ranges  0x0000000000001198      0x148 Middlewares/Third_Party/FreeRTOS/Source/queue.o
 .debug_ranges  0x00000000000012e0      0x1e8 Middlewares/Third_Party/FreeRTOS/Source/tasks.o
 .debug_ranges  0x00000000000014c8       0xd8 Middlewares/Third_Party/FreeRTOS/Source/timers.o
 .debug_ranges  0x00000000000015a0       0x70 Middlewares/Third_Party/FreeRTOS/Source/portable/GCC/ARM_CM4F/port.o
 .debug_ranges  0x0000000000001610       0x40 Middlewares/Third_Party/FreeRTOS/Source/portable/MemMang/heap_4.o

.debug_macro    0x0000000000000000    0x1990d
 .debug_macro   0x0000000000000000      0x2cd Core/Src/GFX_BW.o
 .debug_macro   0x00000000000002cd      0xa5a Core/Src/GFX_BW.o
 .debug_macro   0x0000000000000d27      0x29a Core/Src/GFX_BW.o
 .debug_macro   0x0000000000000fc1       0x2e Core/Src/GFX_BW.o
 .debug_macro   0x0000000000000fef       0x28 Core/Src/GFX_BW.o
 .debug_macro   0x0000000000001017       0x22 Core/Src/GFX_BW.o
 .debug_macro   0x0000000000001039       0x8e Core/Src/GFX_BW.o
 .debug_macro   0x00000000000010c7       0x51 Core/Src/GFX_BW.o
 .debug_macro   0x0000000000001118       0xef Core/Src/GFX_BW.o
 .debug_macro   0x0000000000001207       0x6a Core/Src/GFX_BW.o
 .debug_macro   0x0000000000001271      0x1df Core/Src/GFX_BW.o
 .debug_macro   0x0000000000001450       0x1c Core/Src/GFX_BW.o
 .debug_macro   0x000000000000146c       0x22 Core/Src/GFX_BW.o
 .debug_macro   0x000000000000148e       0xdf Core/Src/GFX_BW.o
 .debug_macro   0x000000000000156d     0x102d Core/Src/GFX_BW.o
 .debug_macro   0x000000000000259a      0x11f Core/Src/GFX_BW.o
 .debug_macro   0x00000000000026b9     0xb937 Core/Src/GFX_BW.o
 .debug_macro   0x000000000000dff0       0x43 Core/Src/GFX_BW.o
 .debug_macro   0x000000000000e033     0x3659 Core/Src/GFX_BW.o
 .debug_macro   0x000000000001168c      0x174 Core/Src/GFX_BW.o
 .debug_macro   0x0000000000011800       0x5a Core/Src/GFX_BW.o
 .debug_macro   0x000000000001185a      0x447 Core/Src/GFX_BW.o
 .debug_macro   0x0000000000011ca1      0x9fe Core/Src/GFX_BW.o
 .debug_macro   0x000000000001269f      0x117 Core/Src/GFX_BW.o
 .debug_macro   0x00000000000127b6      0x11b Core/Src/GFX_BW.o
 .debug_macro   0x00000000000128d1       0x27 Core/Src/GFX_BW.o
 .debug_macro   0x00000000000128f8      0x15f Core/Src/GFX_BW.o
 .debug_macro   0x0000000000012a57      0x287 Core/Src/GFX_BW.o
 .debug_macro   0x0000000000012cde       0x5f Core/Src/GFX_BW.o
 .debug_macro   0x0000000000012d3d      0x236 Core/Src/GFX_BW.o
 .debug_macro   0x0000000000012f73      0x132 Core/Src/GFX_BW.o
 .debug_macro   0x00000000000130a5      0x264 Core/Src/GFX_BW.o
 .debug_macro   0x0000000000013309       0x2e Core/Src/GFX_BW.o
 .debug_macro   0x0000000000013337      0x1b5 Core/Src/GFX_BW.o
 .debug_macro   0x00000000000134ec       0x22 Core/Src/GFX_BW.o
 .debug_macro   0x000000000001350e       0xd6 Core/Src/GFX_BW.o
 .debug_macro   0x00000000000135e4      0x11a Core/Src/GFX_BW.o
 .debug_macro   0x00000000000136fe       0x85 Core/Src/GFX_BW.o
 .debug_macro   0x0000000000013783       0x89 Core/Src/GFX_BW.o
 .debug_macro   0x000000000001380c      0x8a0 Core/Src/GFX_BW.o
 .debug_macro   0x00000000000140ac       0x47 Core/Src/GFX_BW.o
 .debug_macro   0x00000000000140f3      0x287 Core/Src/GFX_BW.o
 .debug_macro   0x000000000001437a      0x126 Core/Src/GFX_BW.o
 .debug_macro   0x00000000000144a0       0x58 Core/Src/GFX_BW.o
 .debug_macro   0x00000000000144f8      0x10c Core/Src/GFX_BW.o
 .debug_macro   0x0000000000014604       0x8e Core/Src/GFX_BW.o
 .debug_macro   0x0000000000014692       0x18 Core/Src/GFX_BW.o
 .debug_macro   0x00000000000146aa       0x46 Core/Src/GFX_BW.o
 .debug_macro   0x00000000000146f0       0x3c Core/Src/GFX_BW.o
 .debug_macro   0x000000000001472c       0x34 Core/Src/GFX_BW.o
 .debug_macro   0x0000000000014760       0x16 Core/Src/GFX_BW.o
 .debug_macro   0x0000000000014776       0x35 Core/Src/GFX_BW.o
 .debug_macro   0x00000000000147ab       0x52 Core/Src/GFX_BW.o
 .debug_macro   0x00000000000147fd       0x1f Core/Src/GFX_BW.o
 .debug_macro   0x000000000001481c       0x43 Core/Src/GFX_BW.o
 .debug_macro   0x000000000001485f       0x20 Core/Src/GFX_BW.o
 .debug_macro   0x000000000001487f      0x1a3 Core/Src/GFX_BW.o
 .debug_macro   0x0000000000014a22      0x32a Core/Src/GFX_BW.o
 .debug_macro   0x0000000000014d4c       0x16 Core/Src/GFX_BW.o
 .debug_macro   0x0000000000014d62       0x29 Core/Src/GFX_BW.o
 .debug_macro   0x0000000000014d8b      0x2c0 Core/Src/SSD1306_OLED.o
 .debug_macro   0x000000000001504b       0x10 Core/Src/SSD1306_OLED.o
 .debug_macro   0x000000000001505b       0x20 Core/Src/SSD1306_OLED.o
 .debug_macro   0x000000000001507b      0x1ff Core/Src/bmp280.o
 .debug_macro   0x000000000001527a      0x130 Core/Src/bmp280.o
 .debug_macro   0x00000000000153aa      0x2e2 Core/Src/freertos.o
 .debug_macro   0x000000000001568c      0x137 Core/Src/freertos.o
 .debug_macro   0x00000000000157c3      0x15a Core/Src/freertos.o
 .debug_macro   0x000000000001591d       0xc9 Core/Src/freertos.o
 .debug_macro   0x00000000000159e6       0x1c Core/Src/freertos.o
 .debug_macro   0x0000000000015a02       0x26 Core/Src/freertos.o
 .debug_macro   0x0000000000015a28      0x4b0 Core/Src/freertos.o
 .debug_macro   0x0000000000015ed8       0xb5 Core/Src/freertos.o
 .debug_macro   0x0000000000015f8d       0xaa Core/Src/freertos.o
 .debug_macro   0x0000000000016037       0x6c Core/Src/freertos.o
 .debug_macro   0x00000000000160a3       0x74 Core/Src/freertos.o
 .debug_macro   0x0000000000016117       0xdd Core/Src/freertos.o
 .debug_macro   0x00000000000161f4       0x58 Core/Src/freertos.o
 .debug_macro   0x000000000001624c       0x22 Core/Src/freertos.o
 .debug_macro   0x000000000001626e       0x10 Core/Src/freertos.o
 .debug_macro   0x000000000001627e      0x200 Core/Src/gpio.o
 .debug_macro   0x000000000001647e      0x200 Core/Src/i2c.o
 .debug_macro   0x000000000001667e      0x2a8 Core/Src/main.o
 .debug_macro   0x0000000000016926      0x137 Core/Src/main.o
 .debug_macro   0x0000000000016a5d       0x66 Core/Src/main.o
 .debug_macro   0x0000000000016ac3      0x10e Core/Src/printf.o
 .debug_macro   0x0000000000016bd1       0x22 Core/Src/printf.o
 .debug_macro   0x0000000000016bf3      0x201 Core/Src/printf.o
 .debug_macro   0x0000000000016df4      0x1f6 Core/Src/stm32f4xx_hal_msp.o
 .debug_macro   0x0000000000016fea      0x1e7 Core/Src/stm32f4xx_hal_timebase_tim.o
 .debug_macro   0x00000000000171d1      0x200 Core/Src/stm32f4xx_it.o
 .debug_macro   0x00000000000173d1      0x1ed Core/Src/system_stm32f4xx.o
 .debug_macro   0x00000000000175be      0x200 Core/Src/usart.o
 .debug_macro   0x00000000000177be      0x247 Drivers/STM32F4xx_HAL_Driver/Src/stm32f4xx_hal.o
 .debug_macro   0x0000000000017a05      0x1e7 Drivers/STM32F4xx_HAL_Driver/Src/stm32f4xx_hal_cortex.o
 .debug_macro   0x0000000000017bec      0x21d Drivers/STM32F4xx_HAL_Driver/Src/stm32f4xx_hal_gpio.o
 .debug_macro   0x0000000000017e09      0x22e Drivers/STM32F4xx_HAL_Driver/Src/stm32f4xx_hal_i2c.o
 .debug_macro   0x0000000000018037      0x20b Drivers/STM32F4xx_HAL_Driver/Src/stm32f4xx_hal_rcc.o
 .debug_macro   0x0000000000018242      0x1e8 Drivers/STM32F4xx_HAL_Driver/Src/stm32f4xx_hal_tim.o
 .debug_macro   0x000000000001842a      0x1e7 Drivers/STM32F4xx_HAL_Driver/Src/stm32f4xx_hal_tim_ex.o
 .debug_macro   0x0000000000018611      0x1e8 Drivers/STM32F4xx_HAL_Driver/Src/stm32f4xx_hal_uart.o
 .debug_macro   0x00000000000187f9      0x23a Middlewares/Third_Party/FreeRTOS/Source/CMSIS_RTOS_V2/cmsis_os2.o
 .debug_macro   0x0000000000018a33       0x10 Middlewares/Third_Party/FreeRTOS/Source/CMSIS_RTOS_V2/cmsis_os2.o
 .debug_macro   0x0000000000018a43       0xd3 Middlewares/Third_Party/FreeRTOS/Source/CMSIS_RTOS_V2/cmsis_os2.o
 .debug_macro   0x0000000000018b16       0x91 Middlewares/Third_Party/FreeRTOS/Source/CMSIS_RTOS_V2/cmsis_os2.o
 .debug_macro   0x0000000000018ba7       0x8d Middlewares/Third_Party/FreeRTOS/Source/CMSIS_RTOS_V2/cmsis_os2.o
 .debug_macro   0x0000000000018c34       0x9a Middlewares/Third_Party/FreeRTOS/Source/CMSIS_RTOS_V2/cmsis_os2.o
 .debug_macro   0x0000000000018cce      0x17a Middlewares/Third_Party/FreeRTOS/Source/list.o
 .debug_macro   0x0000000000018e48      0x209 Middlewares/Third_Party/FreeRTOS/Source/queue.o
 .debug_macro   0x0000000000019051       0x16 Middlewares/Third_Party/FreeRTOS/Source/queue.o
 .debug_macro   0x0000000000019067       0x87 Middlewares/Third_Party/FreeRTOS/Source/queue.o
 .debug_macro   0x00000000000190ee      0x272 Middlewares/Third_Party/FreeRTOS/Source/tasks.o
 .debug_macro   0x0000000000019360       0x10 Middlewares/Third_Party/FreeRTOS/Source/tasks.o
 .debug_macro   0x0000000000019370      0x1cf Middlewares/Third_Party/FreeRTOS/Source/timers.o
 .debug_macro   0x000000000001953f       0x97 Middlewares/Third_Party/FreeRTOS/Source/timers.o
 .debug_macro   0x00000000000195d6      0x196 Middlewares/Third_Party/FreeRTOS/Source/portable/GCC/ARM_CM4F/port.o
 .debug_macro   0x000000000001976c      0x1a1 Middlewares/Third_Party/FreeRTOS/Source/portable/MemMang/heap_4.o

.debug_line     0x0000000000000000    0x1405b
 .debug_line    0x0000000000000000      0xb49 Core/Src/GFX_BW.o
 .debug_line    0x0000000000000b49      0x8e2 Core/Src/SSD1306_OLED.o
 .debug_line    0x000000000000142b      0x803 Core/Src/bmp280.o
 .debug_line    0x0000000000001c2e      0x97b Core/Src/freertos.o
 .debug_line    0x00000000000025a9      0x6ef Core/Src/gpio.o
 .debug_line    0x0000000000002c98      0x718 Core/Src/i2c.o
 .debug_line    0x00000000000033b0      0x8b2 Core/Src/main.o
 .debug_line    0x0000000000003c62      0x94d Core/Src/printf.o
 .debug_line    0x00000000000045af      0x6e7 Core/Src/stm32f4xx_hal_msp.o
 .debug_line    0x0000000000004c96      0x71a Core/Src/stm32f4xx_hal_timebase_tim.o
 .debug_line    0x00000000000053b0      0x76c Core/Src/stm32f4xx_it.o
 .debug_line    0x0000000000005b1c      0x701 Core/Src/system_stm32f4xx.o
 .debug_line    0x000000000000621d      0x71a Core/Src/usart.o
 .debug_line    0x0000000000006937       0x85 Core/Startup/startup_stm32f411retx.o
 .debug_line    0x00000000000069bc      0x8eb Drivers/STM32F4xx_HAL_Driver/Src/stm32f4xx_hal.o
 .debug_line    0x00000000000072a7      0xa0f Drivers/STM32F4xx_HAL_Driver/Src/stm32f4xx_hal_cortex.o
 .debug_line    0x0000000000007cb6      0x88e Drivers/STM32F4xx_HAL_Driver/Src/stm32f4xx_hal_gpio.o
 .debug_line    0x0000000000008544     0x1b99 Drivers/STM32F4xx_HAL_Driver/Src/stm32f4xx_hal_i2c.o
 .debug_line    0x000000000000a0dd      0x943 Drivers/STM32F4xx_HAL_Driver/Src/stm32f4xx_hal_rcc.o
 .debug_line    0x000000000000aa20     0x17a8 Drivers/STM32F4xx_HAL_Driver/Src/stm32f4xx_hal_tim.o
 .debug_line    0x000000000000c1c8      0xcf6 Drivers/STM32F4xx_HAL_Driver/Src/stm32f4xx_hal_tim_ex.o
 .debug_line    0x000000000000cebe      0xff9 Drivers/STM32F4xx_HAL_Driver/Src/stm32f4xx_hal_uart.o
 .debug_line    0x000000000000deb7     0x1e11 Middlewares/Third_Party/FreeRTOS/Source/CMSIS_RTOS_V2/cmsis_os2.o
 .debug_line    0x000000000000fcc8      0x65d Middlewares/Third_Party/FreeRTOS/Source/list.o
 .debug_line    0x0000000000010325     0x10f2 Middlewares/Third_Party/FreeRTOS/Source/queue.o
 .debug_line    0x0000000000011417     0x13fa Middlewares/Third_Party/FreeRTOS/Source/tasks.o
 .debug_line    0x0000000000012811      0xa70 Middlewares/Third_Party/FreeRTOS/Source/timers.o
 .debug_line    0x0000000000013281      0x697 Middlewares/Third_Party/FreeRTOS/Source/portable/GCC/ARM_CM4F/port.o
 .debug_line    0x0000000000013918      0x743 Middlewares/Third_Party/FreeRTOS/Source/portable/MemMang/heap_4.o

.debug_str      0x0000000000000000    0x99d0a
 .debug_str     0x0000000000000000    0x8a6a9 Core/Src/GFX_BW.o
                                      0x8a9df (size before relaxing)
 .debug_str     0x000000000008a6a9      0x568 Core/Src/SSD1306_OLED.o
                                      0x8aa84 (size before relaxing)
 .debug_str     0x000000000008ac11      0x56f Core/Src/bmp280.o
                                      0x87b56 (size before relaxing)
 .debug_str     0x000000000008b180     0x5264 Core/Src/freertos.o
                                      0x8d3c2 (size before relaxing)
 .debug_str     0x00000000000903e4      0x188 Core/Src/gpio.o
                                      0x872a6 (size before relaxing)
 .debug_str     0x000000000009056c       0x71 Core/Src/i2c.o
                                      0x877ab (size before relaxing)
 .debug_str     0x00000000000905dd      0x329 Core/Src/main.o
                                      0x8c3ed (size before relaxing)
 .debug_str     0x0000000000090906      0x997 Core/Src/printf.o
                                       0x4b79 (size before relaxing)
 .debug_str     0x000000000009129d      0x3b8 Core/Src/stm32f4xx_hal_msp.o
                                      0x8759f (size before relaxing)
 .debug_str     0x0000000000091655       0xab Core/Src/stm32f4xx_hal_timebase_tim.o
                                      0x87989 (size before relaxing)
 .debug_str     0x0000000000091700       0xab Core/Src/stm32f4xx_it.o
                                      0x87599 (size before relaxing)
 .debug_str     0x00000000000917ab       0xc4 Core/Src/system_stm32f4xx.o
                                      0x8716a (size before relaxing)
 .debug_str     0x000000000009186f       0x57 Core/Src/usart.o
                                      0x876e6 (size before relaxing)
 .debug_str     0x00000000000918c6       0x36 Core/Startup/startup_stm32f411retx.o
                                         0x82 (size before relaxing)
 .debug_str     0x00000000000918fc      0x542 Drivers/STM32F4xx_HAL_Driver/Src/stm32f4xx_hal.o
                                      0x87adf (size before relaxing)
 .debug_str     0x0000000000091e3e      0x389 Drivers/STM32F4xx_HAL_Driver/Src/stm32f4xx_hal_cortex.o
                                      0x878bc (size before relaxing)
 .debug_str     0x00000000000921c7      0x20c Drivers/STM32F4xx_HAL_Driver/Src/stm32f4xx_hal_gpio.o
                                      0x873a9 (size before relaxing)
 .debug_str     0x00000000000923d3      0xab0 Drivers/STM32F4xx_HAL_Driver/Src/stm32f4xx_hal_i2c.o
                                      0x880ca (size before relaxing)
 .debug_str     0x0000000000092e83      0x239 Drivers/STM32F4xx_HAL_Driver/Src/stm32f4xx_hal_rcc.o
                                      0x87557 (size before relaxing)
 .debug_str     0x00000000000930bc      0xd69 Drivers/STM32F4xx_HAL_Driver/Src/stm32f4xx_hal_tim.o
                                      0x88264 (size before relaxing)
 .debug_str     0x0000000000093e25      0x4ec Drivers/STM32F4xx_HAL_Driver/Src/stm32f4xx_hal_tim_ex.o
                                      0x87a64 (size before relaxing)
 .debug_str     0x0000000000094311      0x50d Drivers/STM32F4xx_HAL_Driver/Src/stm32f4xx_hal_uart.o
                                      0x879a4 (size before relaxing)
 .debug_str     0x000000000009481e     0x27d2 Middlewares/Third_Party/FreeRTOS/Source/CMSIS_RTOS_V2/cmsis_os2.o
                                       0xe365 (size before relaxing)
 .debug_str     0x0000000000096ff0      0x12d Middlewares/Third_Party/FreeRTOS/Source/list.o
                                       0xa686 (size before relaxing)
 .debug_str     0x000000000009711d      0x925 Middlewares/Third_Party/FreeRTOS/Source/queue.o
                                       0xbfe5 (size before relaxing)
 .debug_str     0x0000000000097a42     0x1269 Middlewares/Third_Party/FreeRTOS/Source/tasks.o
                                       0xcb1c (size before relaxing)
 .debug_str     0x0000000000098cab      0x60b Middlewares/Third_Party/FreeRTOS/Source/timers.o
                                       0xc562 (size before relaxing)
 .debug_str     0x00000000000992b6      0x803 Middlewares/Third_Party/FreeRTOS/Source/portable/GCC/ARM_CM4F/port.o
                                       0x844f (size before relaxing)
 .debug_str     0x0000000000099ab9      0x251 Middlewares/Third_Party/FreeRTOS/Source/portable/MemMang/heap_4.o
                                       0xae79 (size before relaxing)

.comment        0x0000000000000000       0x7b
 .comment       0x0000000000000000       0x7b Core/Src/GFX_BW.o
                                         0x7c (size before relaxing)
 .comment       0x000000000000007b       0x7c Core/Src/SSD1306_OLED.o
 .comment       0x000000000000007b       0x7c Core/Src/bmp280.o
 .comment       0x000000000000007b       0x7c Core/Src/freertos.o
 .comment       0x000000000000007b       0x7c Core/Src/gpio.o
 .comment       0x000000000000007b       0x7c Core/Src/i2c.o
 .comment       0x000000000000007b       0x7c Core/Src/main.o
 .comment       0x000000000000007b       0x7c Core/Src/printf.o
 .comment       0x000000000000007b       0x7c Core/Src/stm32f4xx_hal_msp.o
 .comment       0x000000000000007b       0x7c Core/Src/stm32f4xx_hal_timebase_tim.o
 .comment       0x000000000000007b       0x7c Core/Src/stm32f4xx_it.o
 .comment       0x000000000000007b       0x7c Core/Src/system_stm32f4xx.o
 .comment       0x000000000000007b       0x7c Core/Src/usart.o
 .comment       0x000000000000007b       0x7c Drivers/STM32F4xx_HAL_Driver/Src/stm32f4xx_hal.o
 .comment       0x000000000000007b       0x7c Drivers/STM32F4xx_HAL_Driver/Src/stm32f4xx_hal_cortex.o
 .comment       0x000000000000007b       0x7c Drivers/STM32F4xx_HAL_Driver/Src/stm32f4xx_hal_gpio.o
 .comment       0x000000000000007b       0x7c Drivers/STM32F4xx_HAL_Driver/Src/stm32f4xx_hal_i2c.o
 .comment       0x000000000000007b       0x7c Drivers/STM32F4xx_HAL_Driver/Src/stm32f4xx_hal_rcc.o
 .comment       0x000000000000007b       0x7c Drivers/STM32F4xx_HAL_Driver/Src/stm32f4xx_hal_tim.o
 .comment       0x000000000000007b       0x7c Drivers/STM32F4xx_HAL_Driver/Src/stm32f4xx_hal_tim_ex.o
 .comment       0x000000000000007b       0x7c Drivers/STM32F4xx_HAL_Driver/Src/stm32f4xx_hal_uart.o
 .comment       0x000000000000007b       0x7c Middlewares/Third_Party/FreeRTOS/Source/CMSIS_RTOS_V2/cmsis_os2.o
 .comment       0x000000000000007b       0x7c Middlewares/Third_Party/FreeRTOS/Source/list.o
 .comment       0x000000000000007b       0x7c Middlewares/Third_Party/FreeRTOS/Source/queue.o
 .comment       0x000000000000007b       0x7c Middlewares/Third_Party/FreeRTOS/Source/tasks.o
 .comment       0x000000000000007b       0x7c Middlewares/Third_Party/FreeRTOS/Source/timers.o
 .comment       0x000000000000007b       0x7c Middlewares/Third_Party/FreeRTOS/Source/portable/GCC/ARM_CM4F/port.o
 .comment       0x000000000000007b       0x7c Middlewares/Third_Party/FreeRTOS/Source/portable/MemMang/heap_4.o

.debug_frame    0x0000000000000000     0x66a4
 .debug_frame   0x0000000000000000      0x33c Core/Src/GFX_BW.o
 .debug_frame   0x000000000000033c       0xe4 Core/Src/SSD1306_OLED.o
 .debug_frame   0x0000000000000420      0x1c8 Core/Src/bmp280.o
 .debug_frame   0x00000000000005e8       0xd8 Core/Src/freertos.o
 .debug_frame   0x00000000000006c0       0x34 Core/Src/gpio.o
 .debug_frame   0x00000000000006f4       0x74 Core/Src/i2c.o
 .debug_frame   0x0000000000000768       0x8c Core/Src/main.o
 .debug_frame   0x00000000000007f4      0x378 Core/Src/printf.o
 .debug_frame   0x0000000000000b6c       0x34 Core/Src/stm32f4xx_hal_msp.o
 .debug_frame   0x0000000000000ba0       0x74 Core/Src/stm32f4xx_hal_timebase_tim.o
 .debug_frame   0x0000000000000c14       0xc4 Core/Src/stm32f4xx_it.o
 .debug_frame   0x0000000000000cd8       0x58 Core/Src/system_stm32f4xx.o
 .debug_frame   0x0000000000000d30       0x74 Core/Src/usart.o
 .debug_frame   0x0000000000000da4      0x374 Drivers/STM32F4xx_HAL_Driver/Src/stm32f4xx_hal.o
 .debug_frame   0x0000000000001118      0x498 Drivers/STM32F4xx_HAL_Driver/Src/stm32f4xx_hal_cortex.o
 .debug_frame   0x00000000000015b0      0x14c Drivers/STM32F4xx_HAL_Driver/Src/stm32f4xx_hal_gpio.o
 .debug_frame   0x00000000000016fc      0xc5c Drivers/STM32F4xx_HAL_Driver/Src/stm32f4xx_hal_i2c.o
 .debug_frame   0x0000000000002358      0x1f0 Drivers/STM32F4xx_HAL_Driver/Src/stm32f4xx_hal_rcc.o
 .debug_frame   0x0000000000002548     0x10e8 Drivers/STM32F4xx_HAL_Driver/Src/stm32f4xx_hal_tim.o
 .debug_frame   0x0000000000003630      0x5c0 Drivers/STM32F4xx_HAL_Driver/Src/stm32f4xx_hal_tim_ex.o
 .debug_frame   0x0000000000003bf0      0x844 Drivers/STM32F4xx_HAL_Driver/Src/stm32f4xx_hal_uart.o
 .debug_frame   0x0000000000004434      0x978 Middlewares/Third_Party/FreeRTOS/Source/CMSIS_RTOS_V2/cmsis_os2.o
 .debug_frame   0x0000000000004dac       0xd8 Middlewares/Third_Party/FreeRTOS/Source/list.o
 .debug_frame   0x0000000000004e84      0x5ec Middlewares/Third_Party/FreeRTOS/Source/queue.o
 .debug_frame   0x0000000000005470      0x8a8 Middlewares/Third_Party/FreeRTOS/Source/tasks.o
 .debug_frame   0x0000000000005d18      0x3dc Middlewares/Third_Party/FreeRTOS/Source/timers.o
 .debug_frame   0x00000000000060f4      0x1a8 Middlewares/Third_Party/FreeRTOS/Source/portable/GCC/ARM_CM4F/port.o
 .debug_frame   0x000000000000629c      0x108 Middlewares/Third_Party/FreeRTOS/Source/portable/MemMang/heap_4.o
 .debug_frame   0x00000000000063a4       0x2c d:/stm32cubeide_1.5.0/stm32cubeide/plugins/com.st.stm32cube.ide.mcu.externaltools.gnu-tools-for-stm32.7-2018-q2-update.win32_1.5.0.202011040924/tools/bin/../lib/gcc/arm-none-eabi/7.3.1/../../../../arm-none-eabi/lib/thumb/v7e-m/fpv4-sp/hard\libc_nano.a(lib_a-init.o)
 .debug_frame   0x00000000000063d0       0x28 d:/stm32cubeide_1.5.0/stm32cubeide/plugins/com.st.stm32cube.ide.mcu.externaltools.gnu-tools-for-stm32.7-2018-q2-update.win32_1.5.0.202011040924/tools/bin/../lib/gcc/arm-none-eabi/7.3.1/../../../../arm-none-eabi/lib/thumb/v7e-m/fpv4-sp/hard\libc_nano.a(lib_a-memcpy-stub.o)
 .debug_frame   0x00000000000063f8       0x20 d:/stm32cubeide_1.5.0/stm32cubeide/plugins/com.st.stm32cube.ide.mcu.externaltools.gnu-tools-for-stm32.7-2018-q2-update.win32_1.5.0.202011040924/tools/bin/../lib/gcc/arm-none-eabi/7.3.1/../../../../arm-none-eabi/lib/thumb/v7e-m/fpv4-sp/hard\libc_nano.a(lib_a-memset.o)
 .debug_frame   0x0000000000006418       0xac d:/stm32cubeide_1.5.0/stm32cubeide/plugins/com.st.stm32cube.ide.mcu.externaltools.gnu-tools-for-stm32.7-2018-q2-update.win32_1.5.0.202011040924/tools/bin/../lib/gcc/arm-none-eabi/7.3.1/thumb/v7e-m/fpv4-sp/hard\libgcc.a(_arm_addsubdf3.o)
 .debug_frame   0x00000000000064c4       0x50 d:/stm32cubeide_1.5.0/stm32cubeide/plugins/com.st.stm32cube.ide.mcu.externaltools.gnu-tools-for-stm32.7-2018-q2-update.win32_1.5.0.202011040924/tools/bin/../lib/gcc/arm-none-eabi/7.3.1/thumb/v7e-m/fpv4-sp/hard\libgcc.a(_arm_muldivdf3.o)
 .debug_frame   0x0000000000006514       0xc4 d:/stm32cubeide_1.5.0/stm32cubeide/plugins/com.st.stm32cube.ide.mcu.externaltools.gnu-tools-for-stm32.7-2018-q2-update.win32_1.5.0.202011040924/tools/bin/../lib/gcc/arm-none-eabi/7.3.1/thumb/v7e-m/fpv4-sp/hard\libgcc.a(_arm_cmpdf2.o)
 .debug_frame   0x00000000000065d8       0x24 d:/stm32cubeide_1.5.0/stm32cubeide/plugins/com.st.stm32cube.ide.mcu.externaltools.gnu-tools-for-stm32.7-2018-q2-update.win32_1.5.0.202011040924/tools/bin/../lib/gcc/arm-none-eabi/7.3.1/thumb/v7e-m/fpv4-sp/hard\libgcc.a(_arm_fixdfsi.o)
 .debug_frame   0x00000000000065fc       0x24 d:/stm32cubeide_1.5.0/stm32cubeide/plugins/com.st.stm32cube.ide.mcu.externaltools.gnu-tools-for-stm32.7-2018-q2-update.win32_1.5.0.202011040924/tools/bin/../lib/gcc/arm-none-eabi/7.3.1/thumb/v7e-m/fpv4-sp/hard\libgcc.a(_arm_fixunsdfsi.o)
 .debug_frame   0x0000000000006620       0x24 d:/stm32cubeide_1.5.0/stm32cubeide/plugins/com.st.stm32cube.ide.mcu.externaltools.gnu-tools-for-stm32.7-2018-q2-update.win32_1.5.0.202011040924/tools/bin/../lib/gcc/arm-none-eabi/7.3.1/thumb/v7e-m/fpv4-sp/hard\libgcc.a(_arm_truncdfsf2.o)
 .debug_frame   0x0000000000006644       0x2c d:/stm32cubeide_1.5.0/stm32cubeide/plugins/com.st.stm32cube.ide.mcu.externaltools.gnu-tools-for-stm32.7-2018-q2-update.win32_1.5.0.202011040924/tools/bin/../lib/gcc/arm-none-eabi/7.3.1/thumb/v7e-m/fpv4-sp/hard\libgcc.a(_aeabi_uldivmod.o)
 .debug_frame   0x0000000000006670       0x34 d:/stm32cubeide_1.5.0/stm32cubeide/plugins/com.st.stm32cube.ide.mcu.externaltools.gnu-tools-for-stm32.7-2018-q2-update.win32_1.5.0.202011040924/tools/bin/../lib/gcc/arm-none-eabi/7.3.1/thumb/v7e-m/fpv4-sp/hard\libgcc.a(_udivmoddi4.o)
